:0400000057EF00F0C6
:100008002B002B002B002B002B002B002B002B0090
:100018002B002B002B002B002B002B002B002B0080
:100028002B002B002B002B002B002B002B002B0070
:100038002B002B002B0017582B002B002B002B001C
:10004800725C2B002B002B002B002B002B002B00AD
:100058002B002B002B002B002B002B002B002B0040
:100068002B002B002B002B002B002B002B002B0030
:100078002B002B002B002B002B002B002B002B0020
:100088002B002B002B002B002B002B002B002B0010
:10009800B65A2B002B002B002B002B002B002B001B
:0A00A8002B002B00FF0035EFAEF037
:10F4440000000000001B1B1B1B1B1B1B1B000000E0
:10F4540000030303031818181818181818030303D3
:10F46400030000001F1F1F1F1F00001F1F1F1F1F5F
:10F474001F001F1F1F1F1F1F1F1F1F1F1F1F1F1FB7
:10F484001F8080808080808080C0C0C0C0C0C0C019
:10F49400C0E0E0E0E0E0E0E0E0F0F0F0F0F0F0F018
:10F4A400F0F8F8F8F8F8F8F8F8FCFCFCFCFCFCFCC4
:10F4B400FCFEFEFEFEFEFEFEFEFFFFFFFFFFFFFF63
:10F4C400FF0C12120C000000000609081E1E080999
:10F4D40006040A11110A0A1100040E0E0E1F00047C
:10F4E400001C141B12131212000103070F0703015F
:10F4F4000000110A0406110000000103161C10008C
:10F5040000B076017C7301DA7501A04F01BE5F0182
:10F514002063011A5F01A2760154770150770154E8
:10F524007401F67601FE7601947601EE7601847616
:10F5340001BE67010E6501747601705077000704FF
:10F5440004070080C094D4202000204175747265A3
:10F5540073203A2020445331384232305F62617262
:10F564006B65722E6820204F6E65576972655F6205
:10F5740061726B65722E6820204C43445F3462696B
:10F5840074735F4932432E682055415254315F46AB
:10F59400756E6374696F6E732E680D0A002044697A
:10F5A400726563746F7279203A433A5C4D504C41F2
:10F5B40042585F50726F6A656374735C5F3138469A
:10F5C40032374B34325F4F57535F445331384232F2
:10F5D400305F323032332E580D0A005A65726F2074
:10F5E4002000756E2020202000646575782020009E
:10F5F40074726F6973200071756174726500636958
:10F604006E71202000736978202020005365707487
:10F61400202000444547524545004555524F20207F
:10F62400004F484D20202000504620202020004438
:10F63400726F697465004761756368650043414E84
:10F6440043454C00436865636B2E002050494331A9
:10F65400384632374B3432202B204F5753207365B2
:10F664006E736F7220445331384232302073757296
:10F674002020504F525420524130290D0A0020526C
:10F6840041303D445331384232302C5241343D6C88
:10F6940065642C5241333D5351412C5243363D5401
:10F6A400582055415254310D0A002050726F6A653A
:10F6B4006374203A202031384632374B34325F4F5E
:10F6C40057535F445331384232305F323032330D56
:10F6D4000A00205243333D53434C2C5243343D5390
:10F6E40044412C42502E2E2E425035205242302E70
:10F6F4002E52350D0A0020436F6E6669672020493B
:10F704006E7465726E616C20466F73632036344D7F
:10F71400487A0D0A0020536F75726365203A2020E1
:10F724006D61696E2E63205F323032332D30343197
:10F73400300D0A0020456570726F6D203A204565D2
:10F7440070726F6D5F5049432E680D0A00202020AF
:10F7540020202020202020202020202020000C00F9
:10F7640020002020415454454E54494F4E203A2005
:10F77400466F72E761676520696E6974204545507C
:10F78400524F4D207061722070726F6772616D6D9F
:10F7940065202070656E64616E74206C65206465FC
:10F7A40076656C6F7070656D656E74204170706CF9
:10F7B40069636174696F6E2C0D0A2020202020700B
:10F7C4006F7572206576697465722020756E652088
:10F7D40072657361697369652073797374656D61AA
:10F7E4007469717565206465732049442320E020A1
:10F7F4006368617175652072656368617267656DC0
:10F80400656E742064652070726F6772616D6D65DA
:10F814000D0A0020506172616D6574726573206514
:10F824006E20456570726F6D2072657374697475AE
:10F83400E973204F4B206574207472616E7366E91E
:10F8440072E97320202D3E207461626C652064652A
:10F85400207472617661696C202053454E534F5277
:10F864005F414444524553535B5B5D200D0A0020C5
:10F87400436F6E6E6563746572206C65732033200C
:10F88400736F6E6465732073757220524130206506
:10F89400742061707075692073757220535730201D
:10F8A400706F757220636F6E74696E7565720D0A80
:10F8B4000020436F6D70696C65206C652025732092
:10F8C40061202573205554430D0A20617665632019
:10F8D40076657273696F6E20584338203A2020256C
:10F8E40064206574205041434B2025730D0A002089
:10F8F400415454454E54494F4E0D0A2020536169DA
:10F90400736965206F626C696761746F69726520E1
:10F914006465732033202049442320736F6E64652B
:10F924007320445331384232300D0A002054657339
:10F9340074207072E973656E6365206427756E20A8
:10F944007365756C2063617074657572204F2E57F2
:10F954002E532E20E0206C6120666F69732073752E
:10F9640072205241300D0A00206170707569207355
:10F9740075722053573020706F7572207265636FF3
:10F984006D6D656E636572206F75205357342070FA
:10F994006F75722076616C696465720D0A0020438C
:10F9A4006F6E6E6563746572206C6120534F4E44B4
:10F9B4004520322C207365756C65202C7075697335
:10F9C40020617070756920737572205357300D0A69
:10F9D4000020436F6E6E6563746572206C61205302
:10F9E4004F4E44452033207365756C65202C70752B
:10F9F4006973206170707569207375722053573074
:10FA04000D0A000D0A2031207365756C2063617046
:10FA140074657572204453313842323020646F6902
:10FA240074206574726520636F6E6E656374E90D8E
:10FA34000A00200D0A53657175656E63652064279D
:10FA4400496E6974204C43442032783136207669FB
:10FA540061204932433120504346383537340D0A4A
:10FA640000204020646563696D616C202325347532
:10FA74002020736F6974204044657669636520377C
:10FA840062697473203D2030582530325820004478
:10FA94006174613A2046616D696C79436F646520D5
:10FAA4002E2E2049442E3D207878787878787878FE
:10FAB40078787878204352433D202E2E0020436FDF
:10FAC4006E6E6563746572206C6120534F4E4445BD
:10FAD4002023312C20707569732061707075692042
:10FAE400737572205357300D0A00204368617267A2
:10FAF400656D656E742063617261637465726573AC
:10FB040020537065636961757820736574202331AF
:10FB14000D0A002025303564202074656D70233172
:10FB24002E20455854455249455552203D202535EF
:10FB34002E33662025632043200900205465737406
:10FB44002070726573656E636520646576696365AC
:10FB540073207375722042757320493243310D0A44
:10FB640000202052656C656374757265206574208D
:10FB74007669737520636F6E74656E752045657064
:10FB8400726F6D0D0A002074656D7023322E20494A
:10FB94004E54455249455552203D2025352E336655
:10FBA4002025632043200900206164726573736516
:10FBB400204C43443D20256420736F6974203058E1
:10FBC40025303258200D0A000D0A205361757665E0
:10FBD4002049442320736F6E646573204453313885
:10FBE400423230200D0A00202053656E736F72205C
:10FBF400547970652C2049442332202C20435243ED
:10FC040020203A0D0A00202053656E736F72205431
:10FC14007970652C2049442333202C2043524320FF
:10FC2400203A0D0A002074656D7023332E2045415F
:10FC34005520203D2025352E336620256320432082
:10FC44000D0A00202053656E736F7220547970651D
:10FC54002C20494423202C2043524320203A0D0ACF
:10FC640000200D0A20436F6E666967206574204981
:10FC74006E6974204F6E6520576972650D0A002005
:10FC840052656C6563747572652064617461732078
:10FC9400656570726F6D203A200D0A00204166661A
:10FCA40069636861676520737572204C4344203230
:10FCB400783136200D0A002033204D657375726546
:10FCC400732044533138423230202331203A200DFE
:10FCD4000A0020436F64652046616D696C6C652081
:10FCE4003A20445331384232300D0A002050434602
:10FCF4003837353420666F72204C434420327831D3
:10FD040036636172730020466C61672045657072CA
:10FD14006F6D2040307830303030203D200020524C
:10FD2400656375702049442320736F6E64652023D6
:10FD340032200D0A00205265637570204944232047
:10FD4400736F6E6465202333200D0A002020202069
:10FD5400202020202020202020202020202020209F
:10FD6400005049433138462D4B5F44465020312ED4
:10FD7400362E31323500205265616420666C61672D
:10FD8400204030783030203D200020526573746963
:10FD940074756520736F6E64652049442300504375
:10FDA40046383537344120386269747320492F4FFF
:10FDB400004C43442032313139203278313663618A
:10FDC40072730020466C61672040203078303030F8
:10FDD40030203D00542E494E5445522E20202020E0
:10FDE4002020202000542E45585445522E202020F7
:10FDF400202020202000494423312073656E736F36
:10FE040072202020202000494423322073656E7321
:10FE14006F72202020202000494423332073656E14
:10FE2400736F72202020202000436F6E6E65637410
:10FE34002E6C6573203320202000616E6E756C6516
:10FE4400207061722053573020200076616C696401
:10FE54002070617220202053573420006574206183
:10FE640070707569207375722053573000436F6E3C
:10FE74006E65637420534F4E444520233100436F15
:10FE84006E6E65637420534F4E4445202332004305
:10FE94006F6E6E65637420534F4E444520233300C8
:10FEA400313233343536373839303132333435360C
:10FEB400005043463835373420386269747320491A
:10FEC4004F004142434445464748494A4B4C4D4EF6
:10FED4004F50002D3E337849442044533138423248
:10FEE4003020002050726573656E746174696F6EA2
:10FEF400203A0052657374697475652045657072A3
:10FF04006F6D00454550524F4D2035313262797442
:10FF140065730020435243203D2025303258200D84
:10FF24000A0020496E69745F49324328293B0D0A4F
:10FF340000402030782530345820202D3E200020E9
:10FF4400436F646520536F6E64652023004F4C45F6
:10FF540044205353443133303600204F5753204903
:10FF64004423203D20006E6F6E20726563656E73BE
:10FF7400E900417072203132203230323300205394
:10FF84006F6E64652049442300204F575320494431
:10FF9400203D200052544320445333323331002057
:10FFA40030782530345820200040203078253034F3
:10FFB40058200030393A35353A3036003030302E5A
:10FFC40030302043003078253032582C0025332E31
:10FFD400326620430030782530325800494E4600BE
:10FFE4004E414E00696E66006E616E006C6C73006B
:0CFFF400202E3100253863006C660000F0
:020000040001F9
:10000000600E3901D96F000EDB6F000EDD6F080E38
:10001000DF6F000EDE6F7A0E0001C76FC10EC66F74
:10002000810EE82EFED7C62FFCD7C72FFAD700D0F7
:10003000CFECB1F0000E0001E76F000EE66FE75164
:1000400009E1800EE65DD8A028EF80F02AEF80F06D
:100050002CEF80F041EF80F0800EE625D96E030E84
:10006000E721DA6E000EDF6EE64BE72BE75109E180
:10007000800EE65DD8A03FEF80F041EF80F02CEFDE
:1000800080F0000EE76F000EE66FE75109E1800E89
:10009000E65DD8A04EEF80F050EF80F052EF80F098
:1000A00067EF80F0000EE625D96E030EE721DA6EC9
:1000B000000EDF6EE64BE72BE75109E1800EE65DAF
:1000C000D8A065EF80F067EF80F052EF80F0000E6F
:1000D000E76F000EE66FE75109E1500EE65DD8A02C
:1000E00074EF80F076EF80F078EF80F08DEF80F0A5
:1000F000700EE625D96E020EE721DA6E000EDF6E75
:10010000E64BE72BE75109E1500EE65DD8A08BEFF7
:1001100080F08DEF80F078EF80F0800EE06F030EBE
:10012000E16F000EF06F630EF16F0CECB7F0290E6B
:100130000001C76F960EC66F7F0EE82EFED7C62F42
:10014000FCD7C72FFAD790ECB9F0E70E076EFE0E7A
:10015000086EC5ECB5F0000E0001E76F000EE66F0B
:10016000E75109E1090EE65DD8A0B9EF80F0BBEFD9
:1001700080F0BDEF80F0DCEF80F0D890E635D96EEE
:10018000E735DA6EA60ED926010EDA226F0078FF67
:1001900007F06F0074FF08F0C5ECB5F00001E64B06
:1001A000E72BE75109E1090EE65DD8A0DAEF80F010
:1001B000DCEF80F0BDEF80F090ECB9F0E0C0B6F07D
:1001C000E1C0B7F0B50E0001B86FF80EB96F760E4A
:1001D000BA6FFF0EBB6FB70EBC6FFF0EBD6F090E7F
:1001E000BF6F380EBE6F650EC06FFD0EC16F80EC25
:1001F000B4F0B6C0E4F0B7C0E5F0E0C001F0E1C093
:1002000002F0A7ECB3F090ECB9F0260E076EFF0EEB
:10021000086EC5ECB5F076ECBAF03F0E076EFB0E3B
:10022000086EC5ECB5F084EC9EF090ECB9F0200EB1
:100230005F6E000E0001FB6F100EFA6F700EB66F4E
:10024000020EB76FAC0EB86FFB0EB96F5FC0BAF09D
:10025000BB6B5FC0BCF0BD6B80ECB4F0700E016E88
:10026000020E026EA7ECB3F03D017589360E076EE3
:10027000FA0E086EC5ECB5F03D01738F35ECA7F0B2
:1002800090ECB9F0010EC2ECB2F0010EF0ECB5F05A
:10029000020EC2ECB2F0A00E076EFC0E086EC5ECAA
:1002A000B5F0C60E1F6EFE0E206E4FECB1F0000EC4
:1002B000256E020E246ED5ECADF0090E0001C76F5D
:1002C0001E0EC66FE40EE82EFED7C62FFCD7C72F32
:1002D000FAD700F0A40E1F6EFE0E206E4FECB1F0A8
:1002E000010EF0ECB5F0000E0001E76F000EE66FB6
:1002F000EE0E076EFA0E086EC5ECB5F0000E216E1C
:10030000000E206E010EC2EC98F090ECB9F0000ED9
:10031000026E000E016E97ECBAF00001F16F650EEF
:10032000076EFC0E086EC5ECB5F01CECB8F0660E5E
:10033000076EF70E086EC5ECB5F0650E076EFB0E86
:10034000086EC5ECB5F0010E41EC9DF090ECB9F0F3
:10035000020EF0ECB5F0630E0001F119D8A4B3EF72
:1003600081F0B5EF81F0F2EF81F0170E076EF80E15
:10037000086EC5ECB5F0000E256E010E246ED5ECAE
:10038000ADF0090E0001C76F1E0EC66FE40EE82E19
:10039000FED7C62FFCD7C72FFAD700F0F70E1F6E77
:1003A000FE0E206E4FECB1F0000E256E020E246E94
:1003B000D5ECADF0090E0001C76F1E0EC66FE40E3E
:1003C000E82EFED7C62FFCD7C72FFAD700F0D70EDE
:1003D0001F6EFE0E206E4FECB1F0020EF0ECB5F089
:1003E00011EF85F0F30E076EF80E086EC5ECB5F050
:1003F000300E076EF90E086EC5ECB5F0C10E076E33
:10040000FA0E086EC5ECB5F0000E256E010E246ED6
:10041000D5ECADF0090E0001C76F1E0EC66FE40EDD
:10042000E82EFED7C62FFCD7C72FFAD700F0710EE3
:100430001F6EFE0E206E4FECB1F0000E256E020E08
:10044000246ED5ECADF0090E0001C76F1E0EC66F0D
:10045000E40EE82EFED7C62FFCD7C72FFAD700F040
:10046000600E1F6EFE0E206E4FECB1F0CBB03BEF76
:1004700082F03DEF82F036EF82F0020E0001C76F8E
:10048000A00EC66F920EE82EFED7C62FFCD7C72F40
:10049000FAD700F0CBA04FEF82F051EF82F04AEF95
:1004A00082F03EECBAF0470E076EFC0E086EC5EC0B
:1004B000B5F063ECA8F0000E256E010E246ED5ECAD
:1004C000ADF0090E0001C76F1E0EC66FE40EE82ED8
:1004D000FED7C62FFCD7C72FFAD700F0FA0E1F6E33
:1004E000FD0E206E4FECB1F0000E256E020E246E54
:1004F000D5ECADF0090E0001C76F1E0EC66FE40EFD
:10050000E82EFED7C62FFCD7C72FFAD700F0700E03
:100510000001B66F020EB76FF80EB86FFF0EB96F1D
:100520009A0EBA6F010EBB6F80ECB4F0010E256E0F
:10053000700E266E020E276E020EE0ECBAF0030E6D
:10054000F0ECB5F0CB0E016E010E026E9A0E036E4A
:10055000010E046E000E066E080E056E3EECB5F040
:10056000090E0001F16FAEECA1F0010E41EC9DF01F
:10057000A20E076EF90E086EC5ECB5F0000E256EE2
:10058000010E246ED5ECADF0090E0001C76F1E0EF2
:10059000C66FE40EE82EFED7C62FFCD7C72FFAD7BA
:1005A00000F0820E1F6EFE0E206E4FECB1F0000EBA
:1005B000256E020E246ED5ECADF0090E0001C76F5A
:1005C0001E0EC66FE40EE82EFED7C62FFCD7C72F2F
:1005D000FAD700F0600E1F6EFE0E206E4FECB1F0E9
:1005E000090E0001C76F1E0EC66FE40EE82EFED77F
:1005F000C62FFCD7C72FFAD700F0CBB002EF83F09D
:1006000004EF83F0FDEF82F0020E0001C76FA00E31
:10061000C66F920EE82EFED7C62FFCD7C72FFAD78B
:1006200000F0CBA016EF83F018EF83F011EF83F00A
:10063000010EC2ECB2F0020EC2ECB2F0220E076E56
:10064000FD0E086EC5ECB5F03EECBAF0EB0E076E91
:10065000FB0E086EC5ECB5F063ECA8F0000E256E3D
:10066000010E246ED5ECADF0090E0001C76F1E0E11
:10067000C66FE40EE82EFED7C62FFCD7C72FFAD7D9
:1006800000F00B0E1F6EFE0E206E4FECB1F0000E50
:10069000256E020E246ED5ECADF0090E0001C76F79
:1006A0001E0EC66FE40EE82EFED7C62FFCD7C72F4E
:1006B000FAD700F0700E0001B66F020EB76FF80E99
:1006C000B86FFF0EB96F9A0EBA6F010EBB6F80EC58
:1006D000B4F0010E256E700E266E020E276E020E0D
:1006E000E0ECBAF0030EF0ECB5F06C0E076EF90E0C
:1006F000086EC5ECB5F0000E256E010E246ED5EC2B
:10070000ADF04F0E1F6EFE0E206E4FECB1F0000EDE
:10071000256E020E246ED5ECADF03E0E1F6EFE0E61
:10072000206E4FECB1F0090E0001C76F1E0EC66FB0
:10073000E40EE82EFED7C62FFCD7C72FFAD700F05D
:10074000AFEF83F0020E0001C76FA00EC66F920ECE
:10075000E82EFED7C62FFCD7C72FFAD700F0CBA8BC
:10076000B4EF83F0B6EF83F0BDEF83F0CBB0BBEF17
:1007700083F0BDEF83F0A2EF83F0CBA8C2EF83F04C
:10078000C4EF83F0CDEF83F0CBB0C9EF83F0CBEFB4
:1007900083F0CDEF83F0B8EF82F0D30E016E010E3F
:1007A000026E9A0E036E010E046E000E066E080EA7
:1007B000056E3EECB5F00001F151510FF16FAEEC5A
:1007C000A1F0010E41EC9DF0D50E076EF90E086EFA
:1007D000C5ECB5F0000E256E010E246ED5ECADF023
:1007E000090E0001C76F1E0EC66FE40EE82EFED77D
:1007F000C62FFCD7C72FFAD700F0930E1F6EFE0E40
:10080000206E4FECB1F0000E256E020E246ED5EC7A
:10081000ADF0090E0001C76F1E0EC66FE40EE82E84
:10082000FED7C62FFCD7C72FFAD700F0600E1F6E79
:10083000FE0E206E4FECB1F0090E0001C76F1E0EC8
:10084000C66FE40EE82EFED7C62FFCD7C72FFAD707
:1008500000F0CBB02EEF84F030EF84F029EF84F07D
:10086000020E0001C76FA00EC66F920EE82EFED7D3
:10087000C62FFCD7C72FFAD700F0CBA042EF84F0E9
:1008800044EF84F03DEF84F0010EC2ECB2F0020EB2
:10089000C2ECB2F0390E076EFD0E086EC5ECB5F075
:1008A0003EECBAF00A0E076EFC0E086EC5ECB5F011
:1008B00063ECA8F0000E256E010E246ED5ECADF0B1
:1008C000090E0001C76F1E0EC66FE40EE82EFED79C
:1008D000C62FFCD7C72FFAD700F01C0E1F6EFE0ED6
:1008E000206E4FECB1F0000E256E020E246ED5EC9A
:1008F000ADF0090E0001C76F1E0EC66FE40EE82EA4
:10090000FED7C62FFCD7C72FFAD700F0700E000114
:10091000B66F020EB76FF80EB86FFF0EB96F9A0E72
:10092000BA6F010EBB6F80ECB4F0010E256E700E35
:10093000266E020E276E020EE0ECBAF0030EF0EC0B
:10094000B5F06C0E076EF90E086EC5ECB5F0000E32
:10095000256E010E246ED5ECADF04F0E1F6EFE0E0F
:10096000206E4FECB1F0000E256E020E246ED5EC19
:10097000ADF03E0E1F6EFE0E206E4FECB1F0090E74
:100980000001C76F1E0EC66FE40EE82EFED7C62FFD
:10099000FCD7C72FFAD700F0CFEF84F000F0CBA838
:1009A000D4EF84F0D6EF84F0DDEF84F0CBB0DBEF52
:1009B00084F0DDEF84F0CEEF84F0020E0001C76F0B
:1009C000A00EC66F920EE82EFED7C62FFCD7C72FFB
:1009D000FAD700F0CBA8EFEF84F0F1EF84F0FAEF54
:1009E00084F0CBB0F6EF84F0F8EF84F0FAEF84F007
:1009F000E4EF83F0DB0E016E010E026E9A0E036EC1
:100A0000010E046E000E066E080E056E3EECB5F08B
:100A10000001F151090FF16FAEECA1F0010E41ECB4
:100A20009DF0730E076EF80E086EC5ECB5F0000E63
:100A3000256E010E246ED5ECADF0090E0001C76FD6
:100A40001E0EC66FE40EE82EFED7C62FFCD7C72FAA
:100A5000FAD700F02D0E1F6EFE0E206E4FECB1F097
:100A6000000E256E020E246ED5ECADF0090E0001CD
:100A7000C76F1E0EC66FE40EE82EFED7C62FFCD73A
:100A8000C72FFAD700F0600E1F6EFE0E206E4FECDF
:100A9000B1F0090E0001C76F1E0EC66FE40EE82EFE
:100AA000FED7C62FFCD7C72FFAD700F0CBB05BEF2D
:100AB00085F05DEF85F056EF85F0020E0001C76FFF
:100AC000A00EC66F920EE82EFED7C62FFCD7C72FFA
:100AD000FAD700F0CBA06FEF85F071EF85F06AEFE9
:100AE00085F0010EC2ECB2F0020EC2ECB2F0D80EEC
:100AF0001F6EFD0E206E4FECB1F0000E256E020E43
:100B0000246ED5ECADF0090E0001C76F1E0EC66F46
:100B1000E40EE82EFED7C62FFCD7C72FFAD700F079
:100B2000E90E1F6EFD0E206E4FECB1F0000E0001BD
:100B3000E76F000EE66FBB0E076EFC0E086EC5EC8D
:100B4000B5F03EECBAF0CB0E286E010E296E5FECCC
:100B5000ABF028C0C8F029C0C9F02AC0CAF02BC029
:100B6000CBF0E0C0B6F0E1C0B7F0170E0001B86FEF
:100B7000FB0EB96FE6C0BAF0E7C0BBF0C8C0BCF06E
:100B8000C9C0BDF0CAC0BEF0CBC0BFF0000EC16F7F
:100B9000B00EC06F80ECB4F0E0C001F0E1C002F034
:100BA000A7ECB3F0700E0001B66F020EB76FD10E56
:100BB000B86FFF0EB96FC8C0BAF0C9C0BBF0CAC0E9
:100BC000BCF0CBC0BDF080ECB4F00A0E256E700E08
:100BD000266E020E276E010EE0ECBAF0000E216EBA
:100BE000010E206E000E236E0F0E226E000E246E7C
:100BF0007BECB0F03EECBAF0D30E286E010E296EFD
:100C00005FECABF028C0C8F029C0C9F02AC0CAF018
:100C10002BC0CBF0E0C0B6F0E1C0B7F08A0E000107
:100C2000B86FFB0EB96FC8C0BAF0C9C0BBF0CAC07C
:100C3000BCF0CBC0BDF0000EBF6FB00EBE6F80EC3D
:100C4000B4F0E0C001F0E1C002F0A7ECB3F0700E28
:100C50000001B66F020EB76FD10EB86FFF0EB96FFD
:100C6000C8C0BAF0C9C0BBF0CAC0BCF0CBC0BDF0B0
:100C700080ECB4F00A0E256E700E266E020E276E02
:100C8000020EE0ECBAF0000E216E020E206E000E95
:100C9000236E0F0E226E000E246E7BECB0F03EEC45
:100CA000BAF0DB0E286E010E296E5FECABF028C0A7
:100CB000C8F029C0C9F02AC0CAF02BC0CBF0E0C0F0
:100CC000B6F0E1C0B7F0290E0001B86FFC0EB96FA5
:100CD000C8C0BAF0C9C0BBF0CAC0BCF0CBC0BDF040
:100CE000000EBF6FB00EBE6F80ECB4F0E0C001F03C
:100CF000E1C002F0A7ECB3F0BA780001E64BE72BB5
:100D0000010EF0ECB5F0A1EF85F057EF00F0000E0A
:100D10000001756F000E746F36C086F037C087F023
:100D200038C088F039C089F089BF9BEF86F099EF11
:100D300086F0B1EF86F0000E756F010E746F86C0FD
:100D400001F087C002F088C003F089C004F0ACEC69
:100D5000B8F001C086F002C087F003C088F004C07C
:100D600089F0000E00018D6F000E8C6FCCC078F002
:100D7000CDC079F074517511D8A4C1EF86F0C3EFDE
:100D800086F0CAEF86F0D0A5C8EF86F0CAEF86F0ED
:100D9000E4EF86F074517511D8A4D1EF86F0D3EF4B
:100DA00086F0D9EF86F0000E616F2B0E606FDDEFDD
:100DB00086F0000E616F2D0E606F60C020F28C4BCC
:100DC0008D2B7807D8A0790786C001F087C002F084
:100DD00088C003F089C004F0F1ECA9F0010402100E
:100DE000D8A4F5EF86F0F7EF86F042EF87F0BF0E5C
:100DF0003B6EFF0E3C6E3A503D6E3E6A3B503D26C8
:100E00003C503E223E5007E11A0E3D5CD8B00BEF3D
:100E100087F00DEF87F01CEF87F0200E00018C2586
:100E2000056E020E8D21066EE00E076EFF0E086E37
:100E30004BECB4F029EF87F0200E00018C25056EF5
:100E4000020E8D21066EE80E076EFF0E086E4BEC4B
:100E5000B4F00001FD0E7827FF0E792334C011F0A5
:100E600035C012F0200E136E020E146E78C015F00D
:100E700079C016F010ECADF011C034F012C035F0AE
:100E80008FEF8CF086C001F087C002F088C003F0BD
:100E900089C004F0F1ECA9F001500210D8A453EF7E
:100EA00087F055EF87F089EF87F0BF0E3B6EFF0E9E
:100EB0003C6E3A503D6E3E6A3B503D263C503E22D1
:100EC0003E5007E11A0E3D5CD8B069EF87F06BEF3A
:100ED00087F07AEF87F0200E00018C25056E020E58
:100EE0008D21066EE40E076EFF0E086E4BECB4F01B
:100EF00029EF87F0200E00018C25056E020E8D2152
:100F0000066EEC0E076EFF0E086E4BECB4F029EF88
:100F100087F0000E00018E6F000E8F6F800E906FB5
:100F20003F0E916F000E8B6F000E8A6F86C001F02E
:100F300087C002F088C003F089C004F0000E056E7F
:100F4000000E066E000E076E000E086EE6ECAEF0A8
:100F5000D8B0ADEF87F0AFEF87F032EF88F0CEEF8B
:100F600087F08EC00FF08FC010F090C011F091C0CC
:100F700012F0000E136E000E146E200E156E410E50
:100F8000166ECEEC94F00FC08EF010C08FF011C032
:100F900090F012C091F000018A4B8B2B86C028F094
:100FA00087C029F088C02AF089C02BF0000E136E8C
:100FB000000E146E200E156E410E166E8EC00FF0D0
:100FC0008FC010F090C011F091C012F0CEEC94F0F0
:100FD0000FC02CF010C02DF011C02EF012C02FF059
:100FE0006FECA9F0D8B0F7EF87F0F9EF87F0B1EF29
:100FF00087F019EF88F08EC001F08FC002F090C02A
:1010000003F091C004F0000E056E000E066E200E77
:10101000076E410E086EF5EC96F001C08EF002C02E
:101020008FF003C090F004C091F000018A07D8A0AF
:101030008B0786C028F087C029F088C02AF089C0B5
:101040002BF08EC02CF08FC02DF090C02EF091C0F0
:101050002FF06FECA9F0D8A030EF88F032EF88F0D5
:10106000FBEF87F03AC007F0086A30ECB7F00750A2
:1010700000017B6F7BC07AF0670E7B19D8A443EF29
:1010800088F045EF88F06BEF88F0CE51CF11D8A4EF
:101090004CEF88F04EEF88F052EF88F0000ECF6FE3
:1010A000010ECE6FCFBF5FEF88F0CF5106E1CE05C6
:1010B000D8B05DEF88F05FEF88F065EF88F0000E44
:1010C000776F060E766F74EF88F0CEC076F0CFC0E3
:1010D00077F074EF88F0CFBF70EF88F072EF88F090
:1010E0005FEF88F065EF88F0670E7B19D8A47BEF7F
:1010F00088F07DEF88F0ACEF88F08BAF8BEF88F055
:10110000FC0E8A5DFF0E8B59D8A089EF88F08BEF1B
:1011100088F0AAEF88F0FF0E3B6EFF0E3C6E76C0A3
:101120003DF077C03EF03B503D263C503E228A5178
:101130003D5C3E50800A3F6E8B51800A3F58D8A0DC
:10114000A4EF88F0A6EF88F0AAEF88F0660E7A6F19
:10115000ACEF88F0650E7A6F76C06CF077C06DF0FA
:10116000670E7B19D8A4B7EF88F0B9EF88F0C9EF04
:1011700088F0660E7A19D8A4C0EF88F0C2EF88F024
:10118000CBEF88F08BBFC9EF88F0C7EF88F0CBEFCB
:1011900088F06C4B6D2B660E7A19D8A4D2EF88F0CC
:1011A000D4EF88F0F4EF88F08BBFDBEF88F0D9EF55
:1011B00088F0E7EF88F0000E8E6F000E8F6F800EC4
:1011C000906F3F0E916F000E8B6F000E8A6F670E4F
:1011D0007B19D8B4EEEF88F0F0EF88F0F4EF88F0E8
:1011E0008A516C278B516D23000E856F000E846F22
:1011F00086C07CF087C07DF088C07EF089C07FF01B
:101200008EC06EF08FC06FF090C070F091C071F022
:1012100085EF89F07CC001F07DC002F07EC003F054
:101220007FC004F08EC005F08FC006F090C007F0BC
:1012300091C008F0F5EC96F001C01AF002C01BF066
:1012400003C01CF004C01DF0A3EC9FF01AC080F096
:101250001BC081F01CC082F01DC083F080C001F073
:1012600081C002F082C003F083C004F0ECECA8F06F
:1012700001C072F002C073F07CC028F07DC029F07C
:101280007EC02AF07FC02BF08EC013F08FC014F008
:1012900090C015F091C016F080C00FF081C010F022
:1012A00082C011F083C012F0CEEC94F00FC02CF08D
:1012B00010C02DF011C02EF012C02FF053ECB7F07B
:1012C00028C07CF029C07DF02AC07EF02BC07FF0C2
:1012D0008EC001F08FC002F090C003F091C004F006
:1012E000000E056E000E066E200E076E410E086E93
:1012F000F5EC96F001C08EF002C08FF003C090F0C4
:1013000004C091F00001844B852B6C51845D8551A4
:10131000800A3B6E6D51800A3B58D8A092EF89F04D
:1013200094EF89F00AEF89F08EC00FF08FC010F0B3
:1013300090C011F091C012F0000E136E000E146EEA
:10134000A00E156E400E166ECEEC94F00FC080F01D
:1013500010C081F011C082F012C083F07CC028F070
:101360007DC029F07EC02AF07FC02BF080C02CF019
:1013700081C02DF082C02EF083C02FF06FECA9F059
:10138000D8B0C5EF89F0C7EF89F0D2EF89F0000E31
:101390000001806F000E816F000E826F000E836F60
:1013A000FBEF89F07CC001F07DC002F07EC003F04D
:1013B0007FC004F080C005F081C006F082C007F055
:1013C00083C008F0E6ECAEF0D8A0E9EF89F0EBEFCF
:1013D00089F0FBEF89F0000172B1F1EF89F0F3EFD2
:1013E00089F0FBEF89F0000E806F000E816F000E18
:1013F000826F000E836F86C001F087C002F088C044
:1014000003F089C004F080C005F081C006F082C0FE
:1014100007F083C008F06EEC92F001C07CF002C0CF
:101420007DF003C07EF004C07FF07CC028F07DC05A
:1014300029F07EC02AF07FC02BF0000E136E000E44
:10144000146E200E156E410E166E6EC00FF06FC03A
:1014500010F070C011F071C012F0CEEC94F00FC01B
:101460002CF010C02DF011C02EF012C02FF06FEC38
:10147000A9F0D8A03EEF8AF040EF8AF069EF8AF039
:1014800000018A4B8B2B6EC00FF06FC010F070C044
:1014900011F071C012F0000E136E000E146E200ECB
:1014A000156E410E166ECEEC94F00FC06EF010C0AB
:1014B0006FF011C070F012C071F0660E00017A1961
:1014C000D8A465EF8AF067EF8AF069EF8AF06C4B79
:1014D0006D2B6EC08EF06FC08FF070C090F071C039
:1014E00091F0650E00017A19D8B479EF8AF07BEF9C
:1014F0008AF081EF8AF08AC06AF08BC06BF085EFCA
:101500008AF0000E6B6F000E6A6F000E696F000E9E
:10151000686F000E676F000E666F000E856F000E1D
:10152000846F80EF8BF07CC001F07DC002F07EC044
:1015300003F07FC004F08EC005F08FC006F090C0AD
:1015400007F091C008F0F5EC96F001C01AF002C067
:101550001BF003C01CF004C01DF0A3EC9FF01AC0E8
:1015600080F01BC081F01CC082F01DC083F080C0E1
:1015700001F081C002F082C003F083C004F0ECEC03
:10158000A8F001C072F002C073F00001D0B9CBEF37
:101590008AF0CDEF8AF0EAEF8AF072517311D8A485
:1015A000D4EF8AF0D6EF8AF0EAEF8AF0670E7B1963
:1015B000D8A4DDEF8AF0DFEF8AF0EAEF8AF06BBFA4
:1015C000E6EF8AF0E4EF8AF0EAEF8AF0664B672BE9
:1015D00034EF8BF068516911D8A4F1EF8AF0F3EF82
:1015E0008AF01DEF8BF06BBFFAEF8AF0F8EF8AF00C
:1015F0001DEF8BF0200E8C25D96E020E8D21DA6E38
:101600002E0EDF6E8C4B8D2B7807D8A07907000E3D
:10161000696F010E686F1DEF8BF0200E8C25D96E5F
:10162000020E8D21DA6E300EDF6E8C4B8D2B78071B
:10163000D8A079076607D8A0670766516711D8A4B4
:1016400024EF8BF026EF8BF00DEF8BF0200E8C2526
:10165000D96E020E8D21DA6E7251300FDF6E8C4B17
:101660008D2B7807D8A079077CC028F07DC029F0A1
:101670007EC02AF07FC02BF08EC013F08FC014F014
:1016800090C015F091C016F080C00FF081C010F02E
:1016900082C011F083C012F0CEEC94F00FC02CF099
:1016A00010C02DF011C02EF012C02FF053ECB7F087
:1016B00028C07CF029C07DF02AC07EF02BC07FF0CE
:1016C0008EC001F08FC002F090C003F091C004F012
:1016D000000E056E000E066E200E076E410E086E9F
:1016E000F5EC96F001C08EF002C08FF003C090F0D0
:1016F00004C091F000016A07D8A06B07844B852BCA
:101700006C51845D8551800A3B6E6D51800A3B5857
:10171000D8B08DEF8BF08FEF8BF09DEF8BF08DBFFE
:101720009BEF8BF08D5109E14B0E8C5DD8A09BEFA8
:101730008BF09DEF8BF093EF8AF068516911D8A47C
:10174000A4EF8BF0A6EF8BF0B7EF8BF0D0A9ABEF47
:101750008BF0ADEF8BF0B7EF8BF0200E8C25D96EB0
:10176000020E8D21DA6E2E0EDF6E8C4B8D2B200E2D
:101770008C25D96E020E8D21DA6E000EDF6E650E9D
:101780007A19D8A4C6EF8BF0C8EF8BF02EEF87F054
:10179000000E856F4F0E846F200E8425D96E020EC9
:1017A0008521DA6E000EDF6E000E756F000E746F0D
:1017B0008BBFDFEF8BF0DDEF8BF0E7EF8BF0000EF0
:1017C000756F010E746F8A6D8B1FD8B08B2B000E56
:1017D000776F020E766F18EF8CF08407D8A085071C
:1017E000200E8425D96E020E8521DA6E8AC001F0A2
:1017F0008BC002F0000E046E0A0E036E8EECAEF08B
:101800000150300FDF6E8AC001F08BC002F0000E75
:10181000046E0A0E036E73ECADF001C08AF002C0D4
:101820008BF000017607D8A077077807D8A0790752
:101830008A518B11D8A41FEF8CF021EF8CF0EDEFC3
:101840008BF077BF2EEF8CF0775106E17605D8B09C
:101850002CEF8CF02EEF8CF0EDEF8BF08407D8A0FE
:10186000850774517511D8A438EF8CF03AEF8CF0DD
:1018700040EF8CF0000E636F2B0E626F44EF8CF024
:10188000000E636F2D0E626F200E8425D96E020E3E
:101890008521DA6E60008BF1DFFF7807D8A0790729
:1018A0008407D8A08507BF0E3B6EFF0E3C6E3A50F2
:1018B0003D6E3E6A3B503D263C503E223E5009E183
:1018C0001A0E3D5CD8A067EF8CF069EF8CF06FEFDB
:1018D0008CF0000E656F650E646F73EF8CF0000E78
:1018E000656F450E646F200E8425D96E020E85212A
:1018F000DA6E600093F1DFFF7807D8A07907200E39
:101900008C25056E020E8D21066E200E8425076E35
:10191000020E8521086E4BECB4F02EEF87F012001A
:1019200060000BF1D9FF60000FF1DAFF6F007BFF61
:10193000F6FF6F0077FFF7FF000EF86E0800F55016
:10194000250AD8A4A6EF8CF0A8EF8CF04AEF92F00D
:1019500060000BF1D9FF60000FF1DAFFDE2A000E04
:10196000DD22000E0001CD6F000ECC6FCCC0D0F098
:10197000CDC0D1F0CE69CF69000E9D6F000E9C6F77
:1019800010EF8DF0D08160000BF1D9FF60000FF1F6
:10199000DAFFDE2A000EDD2210EF8DF0D083C3EFD8
:1019A0008CF0D085C3EF8CF0D087C3EF8CF0D0895A
:1019B000C3EF8CF0000E9D6F010E9C6F10EF8DF049
:1019C00060000BF1D9FF60000FF1DAFF6F007BFFC1
:1019D000F6FF6F0077FFF7FF000EF86E0800F55076
:1019E000466E476A4750000AD8B4F9EF8CF0DAEF38
:1019F0008CF04650200AD8B4D4EF8CF0030AD8B447
:101A0000D7EF8CF0080AD8B4D1EF8CF0060AD8B41E
:101A1000C2EF8CF01D0AD8B4CEEF8CF0DAEF8CF068
:101A20009C519D11D8B417EF8DF019EF8DF0E0EFB8
:101A30008CF0D0A11EEF8DF020EF8DF021EF8DF016
:101A4000D09360000BF1D9FF60000FF1DAFF6F0057
:101A50007BFFF6FF6F0077FFF7FF000EF86E0800C0
:101A6000F5502A0AD8A437EF8DF039EF8DF06CEFDE
:101A70008DF060000BF1D9FF60000FF1DAFFDE2A74
:101A8000000EDD22600013F1D9FF600017F1DAFFCC
:101A90006F007CFF46F0020EDE266F007CFF47F0F1
:101AA000000EDD2260001BF1D9FF60001FF1DAFF9C
:101AB0006F0078FFCCF06F0074FFCDF0CDBF65EF05
:101AC0008DF063EF8DF0AEEF8DF0D081CC6DCD1F3A
:101AD000D8B0CD2BAEEF8DF060000BF1D9FF6000D8
:101AE0000FF1DAFF6F0078FF08F06F0074FF09F064
:101AF0001BECA5F008C0CCF009C0CDF089EF8DF04B
:101B000060000BF1D9FF60000FF1DAFFDE2A000E52
:101B1000DD22D00E466EFF0E476E60000BF1D9FF3E
:101B200060000FF1DAFF6F007BFFF6FF6F0077FFB9
:101B3000F7FF000EF86E0800F550486E496A4650EF
:101B4000482647504922495009E10A0E485CD8A06E
:101B5000ACEF8DF0AEEF8DF080EF8DF060000BF10B
:101B6000D9FF60000FF1DAFF6F007BFFF6FF6F0017
:101B700077FFF7FF000EF86E0800F5502E0AD8A484
:101B8000C4EF8DF0C6EF8DF055EF8EF0000E000122
:101B9000CF6F000ECE6F60000BF1D9FF60000FF128
:101BA000DAFFDE2A000EDD2260000BF1D9FF6000B3
:101BB0000FF1DAFF6F007BFFF6FF6F0077FFF7FF93
:101BC000000EF86E0800F5502A0AD8A4EAEF8DF04E
:101BD000ECEF8DF013EF8EF060000BF1D9FF600099
:101BE0000FF1DAFFDE2A000EDD22600013F1D9FFCB
:101BF000600017F1DAFF6F007CFF46F0020EDE2670
:101C00006F007CFF47F0000EDD2260001BF1D9FF62
:101C100060001FF1DAFF6F0078FFCEF06F0074FFF5
:101C2000CFF055EF8EF060000BF1D9FF60000FF19F
:101C3000DAFF6F0078FF08F06F0074FF09F01BEC0B
:101C4000A5F008C0CEF009C0CFF030EF8EF06000F4
:101C50000BF1D9FF60000FF1DAFFDE2A000EDD2262
:101C6000D00E466EFF0E476E60000BF1D9FF60008C
:101C70000FF1DAFF6F007BFFF6FF6F0077FFF7FFD2
:101C8000000EF86E0800F550486E496A4650482626
:101C900047504922495009E10A0E485CD8A053EF49
:101CA0008EF055EF8EF027EF8EF060000BF1D9FF2C
:101CB00060000FF1DAFF6F007BFFF6FF6F0077FF28
:101CC000F7FF000EF86E0800F550076E086A30EC5A
:101CD000B7F007500001AC6FAC51D8B472EF8EF082
:101CE00074EF8EF0BEEF8EF060000BF1D9FF600054
:101CF0000FF1DAFF6F0078FF46F06F0074FF47F0D6
:101D0000010E4626000E472260001BF1F6FF600020
:101D10001FF1F7FF000EF86E0800F550076E086A15
:101D200030ECB7F007500001AD6FAD51D8B49BEF68
:101D30008EF09DEF8EF0BEEF8EF060000BF1D9FFBC
:101D400060000FF1DAFF6F0078FF46F06F0074FF5C
:101D500047F0020E4626000E472260001BF1F6FFF8
:101D600060001FF1F7FF000EF86E0800F550076ED7
:101D7000086A30ECB7F007500001AE6F60000BF15D
:101D8000D9FF60000FF1DAFF6F007BFFF6FF6F00F5
:101D900077FFF7FF000EF86E0800F550630AD8A42D
:101DA000D4EF8EF0D6EF8EF005EF8FF060000BF1E0
:101DB000D9FF60000FF1DAFFDE2A000EDD2260009D
:101DC00013F1D9FF600017F1DAFF6F007CFF46F0D6
:101DD000020EDE266F007CFF47F0000EDD22600061
:101DE0001BF1D9FF60001FF1DAFFDF50AF6F40C079
:101DF0000AF041C00BF0AFC00CF0D0ECABF00AC061
:101E000040F00BC041F06DEF92F060000BF1D9FF94
:101E100060000FF1DAFF6F007BFFF6FF6F0077FFC6
:101E2000F7FF000EF86E0800F550640AD8B41BEFF7
:101E30008FF01DEF8FF035EF8FF060000BF1D9FFC1
:101E400060000FF1DAFF6F007BFFF6FF6F0077FF96
:101E5000F7FF000EF86E0800F550690AD8A433EFBA
:101E60008FF035EF8FF07FEF8FF060000BF1D9FF2F
:101E700060000FF1DAFFDE2A000EDD22600013F1B0
:101E8000D9FF600017F1DAFF6F007CFF46F0020E09
:101E9000DE266F007CFF47F0000EDD2260001BF1A4
:101EA000D9FF60001FF1DAFF6F0078FF92F06F003A
:101EB00074FF93F0000E93BFFF0E946F956F966FB3
:101EC000976F986F996F40C01CF041C01DF092C091
:101ED0001EF093C01FF094C020F095C021F096C072
:101EE00022F097C023F098C024F099C025F079EC37
:101EF0009AF01CC040F01DC041F06DEF92F0660EEC
:101F0000AC19D8A486EF8FF088EF8FF0DBEF8FF05D
:101F100060000BF1D9FF60000FF1DAFF6F007BFF6B
:101F2000F6FF6F0077FFF7FF000EF86E08006F00F6
:101F3000D4FFAFF060000BF1D9FF60000FF1DAFFC2
:101F4000DE2A000EDD22600013F1D9FF600017F1D8
:101F5000DAFF6F007CFF46F0040EDE266F007CFF88
:101F600047F0000EDD2260001BF1D9FF60001FF179
:101F7000DAFF6F0078FFA8F06F0078FFA9F06F001C
:101F800078FFAAF06F0078FFABF040C034F041C09A
:101F900035F0A8C036F0A9C037F0AAC038F0ABC001
:101FA00039F0AFC03AF087EC86F034C040F035C06D
:101FB00041F06DEF92F0AC0E016E000E026EFC0E61
:101FC000036EFF0E046E000E066E020E056E8CECA4
:101FD000A6F001500210D8A4F0EF8FF0F2EF8FF0CE
:101FE00085EF90F060000BF1D9FF60000FF1DAFF90
:101FF0006F0078FF46F06F0074FF47F0010E462631
:10200000000E472260001BF1F6FF60001FF1F7FF92
:10201000000EF86E08006F00D4FFAFF0BF0E466EE2
:10202000FF0E476E60000BF1D9FF60000FF1DAFF81
:102030006F007BFFF6FF6F0077FFF7FF000EF86E73
:102040000800F550486E496A4650482647504922D4
:10205000495007E11A0E485CD8B031EF90F033EFE9
:1020600090F057EF90F0600013F1D9FF600017F186
:10207000DAFF6F007CFF46F0040EDE266F007CFF67
:1020800047F0000EDD2260001BF1D9FF60001FF158
:10209000DAFF6F0078FFA8F06F0078FFA9F06F00FB
:1020A00078FFAAF06F0078FFABF079EF90F0600056
:1020B00013F1D9FF600017F1DAFF6F007CFF46F0E3
:1020C000040EDE266F007CFF47F0000EDD2260006C
:1020D0001BF1D9FF60001FF1DAFF6F0078FFA8F055
:1020E0006F0078FFA9F06F0078FFAAF06F0078FF0B
:1020F000ABF0020E60000BF1D9FF60000FF1DAFFC8
:10210000DE26000EDD22C5EF8FF060000BF1D9FF57
:1021100060000FF1DAFF6F007BFFF6FF6F0077FFC3
:10212000F7FF000EF86E0800F550730AD8B49BEF65
:1021300090F09DEF90F0BCEF90F060000BF1D9FFB4
:1021400060000FF1DAFF6F0078FF01F06F0074FF9D
:1021500002F0F00E036EFF0E046E000E066E030E0C
:10216000056E8CECA6F001500210D8A4BAEF90F0E6
:10217000BCEF90F016EF91F060000BF1D9FF60001A
:102180000FF1DAFF6F007BFFF6FF6F0077FFF7FFBD
:10219000000EF86E0800F550730AD8B4D2EF90F034
:1021A000D4EF90F0DBEF90F0000E00019F6F030E74
:1021B0009E6FE0EF90F0000E00019F6F010E9E6F8A
:1021C00060000BF1D9FF60000FF1DAFF9E51DE26AF
:1021D0009F51DD22600013F1D9FF600017F1DAFF93
:1021E0006F007CFF46F0020EDE266F007CFF47F09A
:1021F000000EDD2260001BF1D9FF60001FF1DAFF45
:102200006F0078FF9AF06F0074FF9BF040C00AF0F7
:1022100041C00BF09AC00CF09BC00DF083ECA3F012
:102220000AC040F00BC041F06DEF92F060000BF17E
:10223000D9FF60000FF1DAFF6F007BFFF6FF6F0040
:1022400077FFF7FF000EF86E0800F550750AD8A466
:102250002CEF91F02EEF91F07AEF91F060000BF1FE
:10226000D9FF60000FF1DAFFDE2A000EDD226000E8
:1022700013F1D9FF600017F1DAFF6F007CFF46F021
:10228000020EDE266F007CFF47F0000EDD226000AC
:102290001BF1D9FF60001FF1DAFF6F0078FF48F0F3
:1022A0006F0074FF49F048C0A0F049C0A1F00001E0
:1022B000A26BA36BA46BA56BA66BA76B40C01CF0B5
:1022C00041C01DF0A0C01EF0A1C01FF0A2C020F0B0
:1022D000A3C021F0A4C022F0A5C023F0A6C024F022
:1022E000A7C025F0ACECA0F01CC040F01DC041F030
:1022F0006DEF92F060000BF1D9FF60000FF1DAFF93
:102300006F007BFFF6FF6F0077FFF7FF000EF86EA0
:102310000800F550780AD8B490EF91F092EF91F060
:10232000AAEF91F060000BF1D9FF60000FF1DAFF26
:102330006F007BFFF6FF6F0077FFF7FF000EF86E70
:102340000800F550580AD8A4A8EF91F0AAEF91F030
:102350000AEF92F060000BF1D9FF60000FF1DAFF95
:102360006F007BFFF6FF6F0077FFF7FF000EF86E40
:1023700008006F00D4FFAFF060000BF1D9FF6000E0
:102380000FF1DAFFDE2A000EDD22600013F1D9FF23
:10239000600017F1DAFF6F007CFF46F0020EDE26C8
:1023A0006F007CFF47F0000EDD2260001BF1D9FFBB
:1023B00060001FF1DAFF6F0078FF48F06F0074FFD4
:1023C00049F048C0A0F049C0A1F00001A26BA36B86
:1023D000A46BA56BA66BA76B40C01CF041C01DF0A1
:1023E000A0C01EF0A1C01FF0A2C020F0A3C021F029
:1023F000A4C022F0A5C023F0A6C024F0A7C025F0F9
:10240000AFC026F0ECEC9BF01CC040F01DC041F0CA
:102410006DEF92F060000BF1D9FF60000FF1DAFF71
:102420006F007BFFF6FF6F0077FFF7FF000EF86E7F
:102430000800F550250AD8A420EF92F022EF92F080
:102440003BEF92F060000BF1D9FF60000FF1DAFF73
:10245000DE2A000EDD22000E026E250E016E40C047
:1024600003F041C004F03CECACF0000E416E010EF4
:10247000406E6DEF92F060000BF1D9FF60000FF13C
:10248000DAFFDE2A000EDD22000E416E000E406EE5
:102490006DEF92F060000BF1D9FF60000FF1DAFFF1
:1024A0006F007BFFF6FF6F0077FFF7FF000EF86EFF
:1024B0000800F550016E026A40C003F041C004F00C
:1024C0003CECACF060000BF1D9FF60000FF1DAFFDB
:1024D000DE2A000EDD2235EF92F012000450800B50
:1024E0000D6E045004240F6E03AE79EF92F07BEF73
:1024F00092F07CEF92F00F800F50D8B482EF92F000
:1025000084EF92F099EF92F00F28D8A48AEF92F01E
:102510008CEF92F094EF92F0000E016E000E026EBE
:10252000000E036E000E046E038E000E046EA1EF0B
:1025300092F0000E016E000E026E000E036E000E91
:10254000046E0850800B0E6E0D500E18D8B4ABEF11
:1025500092F0ADEF92F0AEEF92F00D8C085008249F
:102560000E6E07AEB6EF92F0B8EF92F0B9EF92F0C0
:102570000E800E50D8B4BFEF92F0C1EF92F0D6EFBC
:1025800092F00E28D8A4C7EF92F0C9EF92F0D1EFE5
:1025900092F0000E056E000E066E000E076E000E25
:1025A000086E078E000E086EDEEF92F0000E056ECC
:1025B000000E066E000E076E000E086E0F500E5CC9
:1025C000D8B0E5EF92F0E7EF92F00EEF93F00DAC9C
:1025D000ECEF92F0EEEF92F0F0EF92F0800E0D1A29
:1025E0000FC010F00EC00FF010C00EF001C010F0C0
:1025F00005C001F010C005F002C010F006C002F0E6
:1026000010C006F003C010F007C003F010C007F0C0
:1026100004C010F008C004F010C008F0000E106EE6
:102620000F500EC009F00A6A095E000E0A5A0ABE6F
:1026300023EF93F00A5009E11A0E095CD8A023EFAA
:1026400093F025EF93F05CEF93F00150021003102C
:102650000410D8A42EEF93F031EF93F0010E32EF77
:1026600093F0000E106E000E016E000E026E000E52
:10267000036E000E046E0EC00FF065EF93F010A015
:1026800044EF93F046EF93F04CEF93F0D890103076
:102690000109106E4EEF93F0D890103201A053EF65
:1026A00093F055EF93F056EF93F0108E043404320C
:1026B0000332023201320F2A0E500F5CD8A063EFB2
:1026C00093F065EF93F03FEF93F00DBC6AEF93F05A
:1026D0006CEF93F0ACEF93F00F50D8A472EF93F03F
:1026E00074EF93F07EEF93F0000E016E000E026E19
:1026F000000E036E000E046ECDEF94F0055001261F
:1027000006500222075003220850042204A08BEF37
:1027100093F08DEF93F039EF94F010A092EF93F0D7
:1027200094EF93F09AEF93F0D89010300109106E67
:102730009CEF93F0D890103201A0A1EF93F0A3EF9B
:1027400093F0A4EF93F0108E04340432033202327B
:1027500001320F2A39EF94F00550015C06500258FF
:10276000075003580450800A096E0850800A09581F
:10277000D8B0BDEF93F0BFEF93F0EAEF93F00150C4
:10278000055C096E025006580A6E035007580B6E1E
:10279000045008580C6EFF0E0924016EFF0E0A202B
:1027A000026EFF0E0B20036EFF0E0C20046E800ED7
:1027B0000D1A106C1050D8A4E0EF93F0E2EF93F0F4
:1027C000F2EF93F0010E0126000E022203220422F2
:1027D000F2EF93F00550015E0650025A0750035A7B
:1027E0000850045A0150021003100410D8A4FBEF43
:1027F00093F0FDEF93F032EF94F01050D8A403EF74
:1028000094F005EF94F032EF94F0000E016E000E9C
:10281000026E000E036E000E046ECDEF94F0D890A1
:10282000013602360336043610AE19EF94F01BEF72
:1028300094F01CEF94F0018010A021EF94F023EFAE
:1028400094F027EF94F0D880103629EF94F0D890C8
:1028500010360F50D8B42FEF94F031EF94F032EFE0
:1028600094F00F0603AE37EF94F039EF94F00FEFCA
:1028700094F0000E0E6E10AE40EF94F042EF94F024
:102880005AEF94F010C009F07F0E0916D8B44BEF40
:1028900094F04DEF94F051EF94F0010E0E6E5AEF5C
:1028A00094F001A056EF94F058EF94F05AEF94F0A2
:1028B0004DEF94F00E50D8B460EF94F062EF94F0C6
:1028C0008DEF94F0010E0126000E02220322042255
:1028D00004A06DEF94F06FEF94F08DEF94F001C0D1
:1028E00009F002C00AF003C00BF004C00CF00C3475
:1028F0000C320B320A32093209C001F00AC002F070
:102900000BC003F00CC004F00F28D8B48AEF94F089
:102910008CEF94F08DEF94F00F2A0F28D8B493EF3A
:1029200094F095EF94F09DEF94F00F50D8A49BEFA6
:1029300094F09DEF94F0AFEF94F0000E016E000E56
:10294000026E000E036E000E046E0F50D8A4ABEFA3
:1029500094F0ADEF94F0AFEF94F0000E0D6E0FA079
:10296000B4EF94F0B6EF94F0B9EF94F0038EBAEFB1
:1029700094F0039ED8900F30046E0DAEC2EF94F029
:10298000C4EF94F0C5EF94F0048E01C001F002C0D2
:1029900002F003C003F004C004F012001250800BD8
:1029A0001B6E12501224216E11AED9EF94F0DBEFA2
:1029B00094F0DCEF94F021802150D8B4E2EF94F051
:1029C000E4EF94F0F7EF94F02128D8A4EAEF94F024
:1029D000ECEF94F0F4EF94F0000E0F6E000E106E1A
:1029E000000E116E000E126E118EFFEF94F0000EAD
:1029F0000F6E000E106E000E116E000E126E16504D
:102A0000800B1B1A16501624206E15AE0AEF95F097
:102A10000CEF95F00DEF95F020802050D8B413EF17
:102A200095F015EF95F028EF95F02028D8A41BEF2E
:102A300095F01DEF95F025EF95F0000E136E000E4A
:102A4000146E000E156E000E166E158E30EF95F09A
:102A5000000E136E000E146E000E156E000E166E34
:102A60002050D8B436EF95F038EF95F040EF95F060
:102A70002150D8A43EEF95F040EF95F04AEF95F045
:102A8000000E0F6E000E106E000E116E000E126E14
:102A9000F4EF96F015500F026F00CCFF26F06F0098
:102AA000D0FF27F026501C6E1D6A1E6A1F6A275031
:102AB000226E236A246A256A145010026F00CCFF2C
:102AC00026F06F00D0FF27F026501C26000E1D2296
:102AD0001E221F2227502226000E232224222522D6
:102AE000135011026F00CCFF26F06F00D0FF27F0CB
:102AF00026501C26000E1D221E221F222750222691
:102B0000000E2322242225221EC01FF01DC01EF00D
:102B10001CC01DF01C6A135010026F00CCFF26F081
:102B20006F00D0FF27F026501C2627501D22000ED4
:102B30001E22000E1F2214500F026F00CCFF26F041
:102B40006F00D0FF27F026501C2627501D22000EB4
:102B50001E22000E1F221EC01FF01DC01EF01CC032
:102B60001DF01C6A13500F026F00CCFF26F06F009F
:102B7000D0FF27F026501C2627501D22000E1E22B3
:102B8000000E1F22155010026F00CCFF26F06F00C0
:102B9000D0FF27F02650222627502322000E242281
:102BA000000E2522145011026F00CCFF26F06F009A
:102BB000D0FF27F02650222627502322000E242261
:102BC000000E2522155011026F00CCFF26F06F0079
:102BD000D0FF27F02650176E2750186E196A1A6A10
:102BE00019C01AF018C019F017C018F0176A17505A
:102BF000222618502322195024221A5025221CC0A4
:102C000017F01DC018F01EC019F01FC01AF0190EE1
:102C10000FEF96F0D8901A32193218321732E82E88
:102C20000AEF96F01750222618502322195024221A
:102C30001A5025221EC01FF01DC01EF01CC01DF022
:102C40001C6A205021C017F0186A1726000E18229F
:102C5000820E1724266EFF0E1820276E45EF96F081
:102C6000D89022362336243625361FAE3AEF96F01A
:102C70003CEF96F03DEF96F02280D8901C361D3642
:102C80001E361F362606D8A0270624AE4AEF96F039
:102C90004CEF96F030EF96F0000E206E1FAE53EF23
:102CA00096F055EF96F079EF96F0FF0E1C14176E24
:102CB000FF0E1D14186EFF0E1E14196E7F0E1F14CA
:102CC0001A6E1750181019101A10D8B46AEF96F02F
:102CD0006CEF96F070EF96F0010E206E79EF96F0A3
:102CE00022A075EF96F077EF96F079EF96F06CEF03
:102CF00096F02050D8B47FEF96F081EF96F0A5EFD4
:102D000096F0010E2226000E23222422252225A041
:102D10008CEF96F08EEF96F0A5EF96F022C017F0AC
:102D200023C018F024C019F025C01AF01A341A3242
:102D300019321832173217C022F018C023F019C008
:102D400024F01AC025F0264A272A27BEB0EF96F0B5
:102D5000275008E12628D8A0B0EF96F0B2EF96F001
:102D6000BCEF96F0000E226E000E236E800E246ED5
:102D70007F0E256EEAEF96F027BEC9EF96F027503A
:102D800006E12604D8B0C7EF96F0C9EF96F0D5EF6C
:102D900096F0000E226E000E236E000E246E000EC2
:102DA000256E000E1B6EEAEF96F026C021F0FF0E96
:102DB0002216FF0E23167F0E2416000E251621A0C4
:102DC000E4EF96F0E6EF96F0E7EF96F0248ED890D9
:102DD0002130256E1B50251222C00FF023C010F0A9
:102DE00024C011F025C012F012000450800B116EA7
:102DF00004500424186E03AE00EF97F002EF97F032
:102E000003EF97F018801850D8B409EF97F00BEF44
:102E100097F020EF97F01828D8A411EF97F013EF50
:102E200097F01BEF97F0000E016E000E026E000E81
:102E3000036E000E046E038E000E046E28EF97F0F2
:102E4000000E016E000E026E000E036E000E046E88
:102E50000850800B111A08500824196E07AE33EF82
:102E600097F035EF97F036EF97F019801950D8B4F6
:102E70003CEF97F03EEF97F053EF97F01928D8A466
:102E800044EF97F046EF97F04EEF97F0000E056E87
:102E9000000E066E000E076E000E086E078E000E06
:102EA000086E5BEF97F0000E056E000E066E000ECA
:102EB000076E000E086E0550061007100810D8A403
:102EC00064EF97F066EF97F07EEF97F0000E016EDB
:102ED000000E026E000E036E000E046E800E0312D2
:102EE0007F0E04121150041201C001F002C002F062
:102EF00003C003F004C004F0C1EF98F01850D8A448
:102F000084EF97F086EF97F090EF97F0000E016E48
:102F1000000E026E000E036E000E046EC1EF98F0FC
:102F2000195018C009F00A6A095E000E0A5A7F0E8D
:102F30000924126E000E0A20136E01C00DF002C0AB
:102F40000EF003C00FF004C010F0000E016E000E72
:102F5000026E000E036E000E046E000E146E000E64
:102F6000156E000E166E000E176E000E196EF1EF44
:102F700097F01950D8B4BFEF97F0C1EF97F0D8EFA2
:102F800097F0D8900D360E360F361036D8900136A1
:102F900002360336043617AED0EF97F0D2EF97F033
:102FA000D3EF97F00180D8901436153616361736C1
:102FB00005500D5C06500E5807500F580850105819
:102FC000D8A0E5EF97F0E7EF97F0F0EF97F0178CC8
:102FD00005500D5E06500E5A07500F5A0850105AF1
:102FE000192A190E1964F7EF97F0F9EF97F0B9EF76
:102FF00097F00D500E100F101010D8B402EF98F08B
:1030000004EF98F01CEF98F014801CEF98F0D89023
:10301000013602360336043617AE11EF98F013EF7F
:1030200098F014EF98F00180D890143615361636C3
:1030300017361206D8A0130603AE21EF98F023EF3F
:1030400098F007EF98F0000E196E17AE2AEF98F07F
:103050002CEF98F050EF98F0FF0E1414096EFF0E4D
:1030600015140A6EFF0E16140B6E7F0E17140C6EDD
:1030700009500A100B100C10D8B441EF98F043EF30
:1030800098F047EF98F0010E196E50EF98F001A0FC
:103090004CEF98F04EEF98F050EF98F043EF98F027
:1030A0001950D8B456EF98F058EF98F07CEF98F09C
:1030B000010E0126000E02220322042204A063EF67
:1030C00098F065EF98F07CEF98F001C009F002C02D
:1030D0000AF003C00BF004C00CF00C340C320B32BD
:1030E0000A32093209C001F00AC002F00BC003F035
:1030F0000CC004F0124A132A13BE87EF98F0135045
:1031000008E11228D8A087EF98F089EF98F094EFA3
:1031100098F0000E136E1268000E016E000E026E23
:10312000000E036E000E046E13BEA1EF98F0135054
:1031300006E11204D8B09FEF98F0A1EF98F0AFEF3E
:1031400098F0000E136E000E126E000E016E000E4F
:10315000026E000E036E000E046E000E116E12C0A1
:1031600018F018A0B6EF98F0B8EF98F0BBEF98F011
:10317000038EBCEF98F0039ED8901830046E72EF67
:1031800097F01200266E400EC2ECB2F00D0E236EC8
:103190002D0E226ED80EE82EFED7222EFCD7232E1F
:1031A000FAD72604D8A4D7EF98F0D9EF98F0EBEF30
:1031B00098F0000E026E000E016E000E046E070EF7
:1031C000036E00ECBAF0170E0124076EF60E022013
:1031D000086EC5ECB5F0020E2618D8A4F2EF98F0F0
:1031E000F4EF98F006EF99F0000E026E000E016EFB
:1031F000000E046E070E036E00ECBAF0DF0E012421
:10320000076EF50E0220086EC5ECB5F0030E261809
:10321000D8A40DEF99F00FEF99F021EF99F0000E7F
:10322000026E000E016E000E046E070E036E00ECBF
:10323000BAF0DF0E0124076EF50E0220086EC5EC11
:10324000B5F090ECB9F0000E256E010E246E000E64
:10325000286E000E276E27502810D8B432EF99F050
:1032600034EF99F02DEF9AF0070E2714226E000E1E
:103270002814236E22502310D8A441EF99F043EF75
:1032800099F02DEF9AF02604D8A449EF99F04BEF6E
:1032900099F05DEF99F024C001F025C002F0000E16
:1032A000046E070E036E00ECBAF0170E0124076ED1
:1032B000F60E0220086EC5ECB5F0020E2618D8A452
:1032C00064EF99F066EF99F078EF99F024C001F07F
:1032D00025C002F0000E046E070E036E00ECBAF07B
:1032E000DF0E0124076EF50E0220086EC5ECB5F066
:1032F000030E2618D8A47FEF99F081EF99F093EF91
:1033000099F024C001F025C002F0000E046E070EF3
:10331000036E00ECBAF0DF0E0124076EF50E0220FA
:10332000086EC5ECB5F0244A252A90ECB9F02DEFD3
:103330009AF0C50E2724F66EF40E2820F76EF86A70
:10334000000EF8220800F5500DECB2F02004211018
:10335000D8A4ADEF99F0AFEF99F046EF9AF0C50E13
:103360002724F66EF40E2820F76EF86A000EF82275
:103370000800F55076ECB7F046EF9AF0850E27245A
:10338000F66EF40E2820F76EF86A000EF822080098
:10339000F5500DECB2F020042110D8A4D2EF99F032
:1033A000D4EF99F046EF9AF0850E2724F66EF40ECE
:1033B0002820F76EF86A000EF8220800F55076EC27
:1033C000B7F046EF9AF0450E2724F66EF40E28204B
:1033D000F76EF86A000EF8220800F5500DECB2F016
:1033E00020042110D8A4F7EF99F0F9EF99F046EFF7
:1033F0009AF0450E2724F66EF40E2820F76EF86A30
:10340000000EF8220800F55076ECB7F046EF9AF07F
:10341000C50E2724F66EF40E2820F76EF86A000E0B
:10342000F8220800F5500DECB2F020042110D8A4C9
:103430001CEF9AF01EEF9AF046EF9AF0C50E272483
:10344000F66EF40E2820F76EF86A000EF8220800D7
:10345000F55076ECB7F046EF9AF02650226E236ACC
:103460002350000AD8B437EF9AF008EF9AF02250B0
:10347000010AD8B499EF99F0030AD8B4BEEF99F0D5
:10348000010AD8B4E3EF99F008EF9AF0030E236E27
:10349000080E226E770EE82EFED7222EFCD7232EA2
:1034A000FAD700F020042110D8A459EF9AF05BEF6E
:1034B0009AF05DEF9AF090ECB9F0274A282A28504C
:1034C00009E1400E275CD8A068EF9AF06AEF9AF005
:1034D0002BEF99F0800EC2ECB2F00D0E236E2D0E84
:1034E000226ED80EE82EFED7222EFCD7232EFAD736
:1034F00012001EC036F01FC037F020C038F021C0C7
:1035000039F022C03AF023C03BF024C03CF025C083
:103510003DF03DBE8EEF9AF091EF9AF0010E92EFE2
:103520009AF0000E346E356A34503510D8B49BEFE3
:103530009AF09DEF9AF0ADEF9AF03D1E3C1E3B1EB7
:103540003A1E391E381E371E366C000E37223822BE
:1035500039223A223B223C223D220001CFBFB3EF69
:103560009AF0B5EF9AF0B6EF9AF0D093CFBFC3EFD1
:103570009AF0CF5106E1CE05D8B0C1EF9AF0C3EF73
:103580009AF0C9EF9AF0000E316E010E306ECDEF59
:103590009AF0CEC030F0CFC031F0CCC032F0CDC008
:1035A00033F034503510D8A4D8EF9AF0DAEF9AF00F
:1035B000E1EF9AF0D0A5DFEF9AF0E1EF9AF0E4EFB7
:1035C0009AF03206D8A03306000E3F6E4F0E3E6EC4
:1035D000000E02016F6F69EF9BF03E06D8A03F0618
:1035E000200E3E24D96E020E3F20DA6E36C001F066
:1035F00037C002F038C003F039C004F03AC005F01B
:103600003BC006F03CC007F03DC008F00A0E096E52
:10361000000E0A6E000E0B6E000E0C6E000E0D6E8C
:10362000000E0E6E000E0F6E000E106EDAECA5F09E
:1036300001C026F002C027F003C028F004C029F022
:1036400005C02AF006C02BF007C02CF008C02DF0F2
:1036500026C013F028C014F0DDECB7F01350300F83
:10366000DF6E3006D8A031063206D8A0330636C049
:1036700001F037C002F038C003F039C004F03AC09E
:1036800005F03BC006F03CC007F03DC008F00A0E54
:10369000096E000E0A6E000E0B6E000E0C6E000E10
:1036A0000D6E000E0E6E000E0F6E000E106E57ECBB
:1036B000A4F001C036F002C037F003C038F004C0F7
:1036C00039F005C03AF006C03BF007C03CF008C036
:1036D0003DF03FBE74EF9BF03F5008E13E04D8A0A0
:1036E00074EF9BF076EF9BF0A7EF9BF0365037100E
:1036F000381039103A103B103C103D10D8A483EF1D
:103700009BF085EF9BF0EDEF9AF031BE92EF9BF0CE
:10371000315006E13004D8B090EF9BF092EF9BF06F
:10372000EDEF9AF033BE9DEF9BF0335008E1320489
:10373000D8A09DEF9BF09FEF9BF0A7EF9BF00001BF
:10374000D0B3A5EF9BF0A7EF9BF0EDEF9AF03450CC
:103750003510D8A4AEEF9BF0B0EF9BF0B8EF9BF024
:103760000001D0A5B6EF9BF0B8EF9BF0D7EF9BF030
:103770003E06D8A03F0634503510D8A4C2EF9BF0C7
:10378000C4EF9BF0CAEF9BF0000E2F6E2B0E2E6E37
:10379000CEEF9BF0000E2F6E2D0E2E6E200E3E24CF
:1037A000D96E020E3F20DA6E6000BBF0DFFF1CC056
:1037B00011F01DC012F0200E3E24136E020E3F20A9
:1037C000146E32C015F033C016F010ECADF011C01D
:1037D0001CF012C01DF012000001CFBFF2EF9BF0F1
:1037E000F4EF9BF0F5EF9BF0D093CFBF02EF9CF08E
:1037F000CF5106E1CE05D8B000EF9CF002EF9CF06F
:1038000008EF9CF0000E306E010E2F6E0CEF9CF056
:10381000CEC02FF0CFC030F0CCC031F0CDC032F0F0
:10382000D0A915EF9CF017EF9CF01BEF9CF0FE0E5B
:103830003126FF0E32221EC033F01FC034F020C0EC
:1038400035F021C036F022C037F023C038F024C054
:1038500039F025C03AF0000E3C6E4F0E3B6E000E64
:1038600002016F6FCEEF9CF03B06D8A03C060F0E16
:1038700033143D6E3E6A3EBE47EF9CF03E5009E178
:103880000A0E3D5CD8A047EF9CF049EF9CF051EF49
:103890009CF0570E3D243D6E000E3E203E6E57EFCD
:1038A0009CF0300E3D243D6E000E3E203E6EBF0E5D
:1038B000276EFF0E286E2650296E2A6A2750292669
:1038C00028502A222A5007E11A0E295CD8B06BEF43
:1038D0009CF06DEF9CF090EF9CF09F0E276EFF0E1A
:1038E000286E200E3D10296E000E3E102A6E2750C5
:1038F000292628502A222A5007E11A0E295CD8B01E
:1039000084EF9CF086EF9CF090EF9CF03DC007F0B8
:103910003EC008F099ECB7F007C03DF008C03EF09B
:10392000200E3B24D96E020E3C20DA6E6000F7F0C8
:10393000DFFF2F06D8A030063106D8A0320633C0EC
:1039400027F034C028F035C029F036C02AF037C03F
:103950002BF038C02CF039C02DF03AC02EF0050EF7
:10396000BBEF9CF0D8902E322D322C322B322A32E3
:10397000293228322732E82EB2EF9CF027C033F0EC
:1039800028C034F029C035F02AC036F02BC037F0FB
:103990002CC038F02DC039F02EC03AF03CBEDAEF22
:1039A0009CF03C5009E1020E3B5CD8A0DAEF9CF0A1
:1039B000DCEF9CF00DEF9DF03350341035103610D5
:1039C0003710381039103A10D8A4E9EF9CF0EBEF1B
:1039D0009CF034EF9CF030BEF8EF9CF0305006E1E4
:1039E0002F04D8B0F6EF9CF0F8EF9CF034EF9CF089
:1039F00032BE03EF9DF0325008E13104D8A003EF4E
:103A00009DF005EF9DF00DEF9DF00001D0B30BEFA1
:103A10009DF00DEF9DF034EF9CF00001D0A913EF65
:103A20009DF015EF9DF02CEF9DF03B06D8A03C06D5
:103A3000200E3B24D96E020E3C20DA6E60009BF013
:103A4000DFFF3B06D8A03C06200E3B24D96E020EB9
:103A50003C20DA6E300EDF6E1CC011F01DC012F07B
:103A6000200E3B24136E020E3C20146E31C015F064
:103A700032C016F010ECADF011C01CF012C01DF0F9
:103A800012005D6E000E0001DB6F000EDA6F000E9B
:103A9000D96F000ED86F000E01016B6F000E6A6FB8
:103AA000000E026E000E016E97ECBAF00001EA6F94
:103AB000EAC0F1F0030E5C6E080E5B6E770EE82E26
:103AC000FED75B2EFCD75C2EFAD700F05D04D8A49D
:103AD0006CEF9DF06EEF9DF096EF9DF0830E076EFC
:103AE000FC0E086EC5ECB5F0C70E076EFD0E086E35
:103AF000C5ECB5F0EAC001F0026A000E046E0A0ED1
:103B0000036E73ECADF00150300F87ECBAF0EAC0F1
:103B100001F0026A000E046E0A0E036E8EECAEF027
:103B20000150300F87ECBAF090ECB9F0000E0001B4
:103B3000DB6F000EDA6F5D04D8A4A1EF9DF0A3EF58
:103B40009DF0B1EF9DF0430E076EFF0E086EC5ECC1
:103B5000B5F00001DA51300F87ECBAF03A0E87EC7D
:103B6000BAF0DAC05BF0DBC05CF05B3A5C3AF00EB6
:103B70005C165B500F0B5C12F00E5B16100E5B2494
:103B800001016A6F000E5C206B6F5D04D8A4CBEF5F
:103B90009DF0CDEF9DF0E5EF9DF0700E0001B66F4A
:103BA000020EB76FA30EB86FFF0EB96F6AC1BAF0FD
:103BB0006BC1BBF080ECB4F0700E016E020E026EB1
:103BC000A7ECB3F0090E87ECBAF0000E0001D96F34
:103BD000000ED86FD85101016A25016E0001D9513C
:103BE00001016B21026E97ECBAF00001EA6F030E3F
:103BF0005C6E080E5B6E770EE82EFED75B2EFCD750
:103C00005C2EFAD700F0DAC001F0DBC002F0000E43
:103C1000046E110E036E00ECBAF0000E5B6E040E23
:103C20005C6E01505B2602505C220001D8515B247F
:103C3000D96ED9515C20DA6E6000ABF3DFFF700EF5
:103C4000B66F020EB76FC90EB86FFF0EB96FEAC03C
:103C5000BAF0BB6B80ECB4F0700E016E020E026E17
:103C6000A7ECB3F00001D84BD92BD9BF41EF9EF0A0
:103C7000D95109E1080ED85DD8A041EF9EF043EF7D
:103C80009EF0EAEF9DF0DAC001F0DBC002F0000E1A
:103C9000046E110E036E00ECBAF0000E5B6E040EA3
:103CA0005C6E01505B2602505C220001D8515B24FF
:103CB000D96ED9515C20DA6E000EDF6E5D04D8A497
:103CC00064EF9EF066EF9EF068EF9EF090ECB9F026
:103CD0000001DA4BDB2BDBBF77EF9EF0DB5109E114
:103CE000030EDA5DD8A077EF9EF079EF9EF09BEFA0
:103CF0009DF05D04D8A47FEF9EF081EF9EF083EFEE
:103D00009EF090ECB9F01200800E0001E06F030EFF
:103D1000E16F3D017599738F000E0001C56F020EB2
:103D2000C46FC4C001F0C5C002F0FFECB8F00009D8
:103D3000D8B49DEF9EF09FEF9EF088EF9FF00001BA
:103D4000C535C5315B6EC431E46F5BC0E5F0E0C0E2
:103D5000B6F0E1C0B7F0650EB86FFA0EB96FC4C027
:103D6000BAF0C5C0BBF0E4C0BCF0E5C0BDF080EC6B
:103D7000B4F032EF9FF0E0C00FF0E1C010F0F00EB1
:103D8000116EFC0E126E51ECBAF080EF9FF0700EC7
:103D9000016E020E026EB50E036EFE0E046E35EC61
:103DA000B3F0E0C001F0E1C002F099ECB5F001C061
:103DB000C2F002C0C3F00001C251E025056EC3513C
:103DC000E121066E700E076E020E086E4BECB4F029
:103DD00080EF9FF0E0C00FF0E1C010F0B50E116E63
:103DE000FD0E126E51ECBAF080EF9FF0E0C00FF0C4
:103DF000E1C010F0A20E116EFD0E126E51ECBAF081
:103E000080EF9FF0E0C00FF0E1C010F0510E116E96
:103E1000FF0E126E51ECBAF080EF9FF0E0C00FF091
:103E2000E1C010F0070E116EFF0E126E51ECBAF0E9
:103E300080EF9FF0E0C00FF0E1C010F0980E116E1F
:103E4000FF0E126E51ECBAF080EF9FF0E0C00FF061
:103E5000E1C010F06A0E116EFF0E126E51ECBAF056
:103E600080EF9FF0E4C05BF0E5C05CF05C50000ABE
:103E7000D8B43DEF9FF026EF9FF05B50200AD8B4F6
:103E8000BBEF9EF0010AD8B4BBEF9EF0030AD8B492
:103E9000BBEF9EF0010AD8B4BBEF9EF0040AD8B481
:103EA000BBEF9EF00F0AD8B4C7EF9EF0010AD8B45A
:103EB000C7EF9EF0030AD8B4C7EF9EF01D0AD8B42E
:103EC000EAEF9EF00F0AD8B4F6EF9EF0010AD8B4DC
:103ED000F6EF9EF0030AD8B4F6EF9EF0010AD8B4CC
:103EE000F6EF9EF0070AD8B402EF9FF06B0AD8B441
:103EF0000EEF9FF03F0AD8B41AEF9FF026EF9FF025
:103F0000E0C001F0E1C002F0A7ECB3F090ECB9F032
:103F1000020E0001C425C46F000EC521C56FC5BFC8
:103F20009BEF9FF0C55109E1FC0EC45DD8A09BEF4B
:103F30009FF09DEF9FF091EF9EF03D01739F75897B
:103F400090ECB9F012004AC12AF04BC12BF04CC1E1
:103F50002CF04DC12DF01AC02AF01BC02BF01CC054
:103F60002CF01DC02DF0810E1E6EFF0E1F6E2AC09C
:103F700020F02BC021F02CC022F02DC023F0180E11
:103F8000C7EF9FF0D8902332223221322032E82E20
:103F9000C2EF9FF020501E24286E000E1F20296EB5
:103FA00029BEDCEF9FF0295009E1170E285CD8A04C
:103FB000DCEF9FF0DEEF9FF0E8EF9FF01AC01AF001
:103FC0001BC01BF01CC01CF01DC01DF0ABEFA0F00F
:103FD00029BEEDEF9FF0EFEF9FF05FEFA0F028C05C
:103FE0001EF0FF0E1F6EFF0E206E7F0E216E000E64
:103FF000226E1E66FEEF9FF006EFA0F02234223202
:10400000213220321F321E2EF9EF9FF01FC024F004
:1040100020C025F021C026F022C027F024502A1409
:104020001E6E25502B141F6E26502C14206E275008
:104030002D14216E1E501F1020102110D8A423EF24
:10404000A0F025EFA0F027EFA0F0DEEF9FF02AC050
:104050001EF02BC01FF02CC020F02DC021F0200E30
:1040600037EFA0F0D890213220321F321E32E82ED6
:1040700032EFA0F01E501F1020102110D8B443EFD3
:10408000A0F045EFA0F04DEFA0F024502A262550D7
:104090002B2226502C2227502D22241C1E6E251C3C
:1040A0001F6E261C206E271C216E1E502A161F50C4
:1040B0002B1620502C1621502D16A3EFA0F02AC04D
:1040C0001EF02BC01FF02CC020F02DC021F0200EC0
:1040D0006FEFA0F0D890213220321F321E32E82E2E
:1040E0006AEFA0F01E501F1020102110D8A47BEF03
:1040F000A0F07DEFA0F087EFA0F0000E2A6E000E7A
:104100002B6E000E2C6E000E2D6EA3EFA0F0D8903B
:104110002A341E6E2B341F6E2C34206E2D34216EEB
:104120001E501F1020102110D8B499EFA0F09BEF63
:10413000A0F0A3EFA0F0000E2A6E000E2B6E800EF2
:104140002C6EBF0E2D6E2AC01AF02BC01BF02CC097
:104150001CF02DC01DF012000001CFBFB2EFA0F087
:10416000B4EFA0F0B5EFA0F0D093CFBFC2EFA0F0B6
:10417000CF5106E1CE05D8B0C0EFA0F0C2EFA0F05D
:10418000C8EFA0F0000E2F6E010E2E6ECCEFA0F047
:10419000CEC02EF0CFC02FF0CCC030F0CDC031F06B
:1041A0001EC032F01FC033F020C034F021C035F003
:1041B00022C036F023C037F024C038F025C039F0D3
:1041C000000E3B6E4F0E3A6E000E02016F6F5FEFF6
:1041D000A1F03A06D8A03B06200E3A24D96E020E72
:1041E0003B20DA6E32C001F033C002F034C003F07D
:1041F00035C004F036C005F037C006F038C007F00F
:1042000039C008F00A0E096E000E0A6E000E0B6E21
:10421000000E0C6E000E0D6E000E0E6E000E0F6E78
:10422000000E106EA8ECACF001C026F002C027F022
:1042300003C028F004C029F005C02AF006C02BF006
:1042400007C02CF008C02DF02650300FDF6E2E0670
:10425000D8A02F063006D8A0310632C001F033C0F6
:1042600002F034C003F035C004F036C005F037C0AA
:1042700006F038C007F039C008F00A0E096E000ECB
:104280000A6E000E0B6E000E0C6E000E0D6E000E10
:104290000E6E000E0F6E000E106E70ECAAF001C0D4
:1042A00032F002C033F003C034F004C035F005C072
:1042B00036F006C037F007C038F008C039F03A5081
:1042C0003B10D8B466EFA1F068EFA1F099EFA1F030
:1042D0003250331034103510361037103810391072
:1042E000D8A475EFA1F077EFA1F0E9EFA0F02FBE11
:1042F00084EFA1F02F5006E12E04D8B082EFA1F098
:1043000084EFA1F0E9EFA0F031BE8FEFA1F03150C2
:1043100008E13004D8A08FEFA1F091EFA1F099EF60
:10432000A1F00001D0B397EFA1F099EFA1F0E9EF70
:10433000A0F01CC011F01DC012F0200E3A24136E24
:10434000020E3B20146E30C015F031C016F010EC98
:10435000ADF011C01CF012C01DF01200000E0001E3
:10436000D76F000ED66F000ED56F000ED46F000E03
:104370000101696F000E686FD29ECC0E076EFB0EB6
:10438000086EC5ECB5F00A0E076EFD0E086EC5ECA2
:10439000B5F0000E026E000E016EF1C003F01AECD3
:1043A000B6F0030E5C6E080E5B6E770EE82EFED73D
:1043B0005B2EFCD75C2EFAD700F0F1C001F0026A48
:1043C000000E046E0A0E036E73ECADF00150300F58
:1043D00087ECBAF0F1C001F0026A000E046E0A0E1A
:1043E000036E8EECAEF00150300F87ECBAF090EC1B
:1043F000B9F0000E0001D76F000ED66F820E076E67
:10440000FF0E086EC5ECB5F00001D651300F87ECF9
:10441000BAF0D6C05BF0D7C05CF05B3A5C3AF00E05
:104420005C165B500F0B5C12F00E5B16100E5B24DB
:104430000101686F000E5C20696F700E0001B66F9D
:10444000020EB76F350EB86FFF0EB96F68C1BAF0C4
:1044500069C1BBF080ECB4F0700E016E020E026E0A
:10446000A7ECB3F0000E0001D56F000ED46FD6C0DC
:104470005BF0D7C05CF0D8905B365C36D8905B368A
:104480005C36D8905B365C36CB0E5D6E010E5E6E90
:104490005B505D265C505E22D4515D24D96ED551AF
:1044A0005E20DA6EDF50E96FD45101016825016E9C
:1044B0000001D55101016921026EE9C003F01AEC37
:1044C000B6F0030E5C6E080E5B6E770EE82EFED71C
:1044D0005B2EFCD75C2EFAD700F0700E0001B66F91
:1044E000020EB76FC90EB86FFF0EB96FE9C0BAF010
:1044F000BB6B80ECB4F0700E016E020E026EA7EC86
:10450000B3F00001D44BD52BD5BF90EFA2F0D5511D
:1045100009E1080ED45DD8A090EFA2F092EFA2F0CE
:1045200037EFA2F090ECB9F00001D64BD72BD7BFF4
:10453000A3EFA2F0D75109E1030ED65DD8A0A3EFF7
:10454000A2F0A5EFA2F0FEEFA1F090ECB9F0D28EB0
:104550001200096E0950D8B4B0EFA2F0B2EFA2F089
:10456000D4EFA2F004BEB9EFA2F0B7EFA2F0D4EFFF
:10457000A2F001C005F002C006F003C007F004C0BD
:1045800008F0051E061E071E081E052A000E06223C
:104590000722082205C00BF006C00CF007C00DF082
:1045A00008C00EF0DCEFA2F001C00BF002C00CF06E
:1045B00003C00DF004C00EF00150021003100410EF
:1045C000D8A4E5EFA2F0E7EFA2F0F1EFA2F0000E21
:1045D000016E000E026E000E036E000E046E82EF7E
:1045E000A3F0960E0A6EFBEFA2F00A2AD8900E32C4
:1045F0000D320C320B32000E0B14056E000E0C1433
:10460000066E000E0D14076EFE0E0E14086E055099
:10461000061007100810D8A410EFA3F012EFA3F0B3
:10462000F5EFA2F020EFA3F00A2A010E0B26000EF0
:104630000C220D220E22D8900E320D320C320B328B
:10464000000E0B14056E000E0C14066E000E0D14F9
:10465000076EFF0E0E14086E0550061007100810A6
:10466000D8A435EFA3F037EFA3F014EFA3F03FEF9A
:10467000A3F00A06D8900B360C360D360E360DBE5A
:1046800044EFA3F046EFA3F04EEFA3F0020E0A6052
:104690004CEFA3F04EEFA3F039EFA3F00AB053EFC5
:1046A000A3F055EFA3F056EFA3F00D9ED8900A3279
:1046B0000AC005F0066A076A086A05C008F0076ABA
:1046C000066A056A05500B1206500C1207500D12AF
:1046D00008500E120950D8B470EFA3F072EFA3F097
:1046E0007AEFA3F004BE79EFA3F077EFA3F07AEFAF
:1046F000A3F00E8E0BC001F00CC002F00DC003F051
:104700000EC004F0120020EEC2F110EE0FF0060E03
:104710006F006FFFE3FFE806FBE20CC01AF00DC06C
:104720001BF01A501B10D8A498EFA3F09AEFA3F037
:104730009EEFA3F00F0E1A6E000E1B6E1AC001F052
:104740001BC002F099ECB5F001C01EF002C01FF0D2
:10475000CEC01CF0CFC01DF01DBEB1EFA3F0B3EF73
:10476000A3F0C8EFA3F01E501C5C1D50800A0E6E13
:104770001F50800A0E58D8A0C0EFA3F0C2EFA3F0DC
:10478000C4EFA3F0C8EFA3F01CC01EF01DC01FF0C3
:104790001EC01CF01FC01DF0CCC018F0CDC019F019
:1047A0000001D0B1D6EFA3F0D8EFA3F0F5EFA3F05E
:1047B000E6EFA3F0000E026E200E016E0AC003F0B9
:1047C0000BC004F03CECACF01E4A1F2A18501E5CD3
:1047D0001F50800A0E6E1950800A0E58D8A0F3EFB1
:1047E000A3F0F5EFA3F0DAEFA3F0000E176E000EC2
:1047F000166E1EEFA4F060006BF0F6FF60006FF025
:10480000F7FF000EF86E1F0EF76403D00800F55096
:1048100007D06F00DBFFE9FF6F00DFFFEAFFEF501B
:104820000E6E0E50016E026A0AC003F00BC004F057
:104830003CECACF01A4A1B2A164A172A1C50165C8C
:104840001750800A0E6E1D50800A0E58D8A02BEF0C
:10485000A4F02DEFA4F0FBEFA3F00001D0A133EF03
:10486000A4F035EFA4F052EFA4F043EFA4F0000E53
:10487000026E200E016E0AC003F00BC004F03CEC87
:10488000ACF01E4A1F2A18501E5C1F50800A0E6E84
:104890001950800A0E58D8A050EFA4F052EFA4F09F
:1048A00037EFA4F01EC00AF01FC00BF01200000E7C
:1048B000126E10BE60EFA4F05EEFA4F072EFA4F0F1
:1048C000101E0F1E0E1E0D1E0C1E0B1E0A1E096C46
:1048D000000E0A220B220C220D220E220F22102281
:1048E000010E126E08BE79EFA4F077EFA4F08BEF03
:1048F000A4F0081E071E061E051E041E031E021E2F
:10490000016C000E02220322042205220622072245
:104910000822010E121A20EE13F0070EDE6AE806D6
:10492000FDE209500A100B100C100D100E100F10A4
:104930001010D8B49EEFA4F0A0EFA4F0F2EFA4F012
:10494000010E116EAEEFA4F0D89009360A360B3680
:104950000C360D360E360F361036112A10AEB3EF68
:10496000A4F0B5EFA4F0A4EFA4F0D8901336143659
:10497000153616361736183619361A360950015CB0
:104980000A5002580B5003580C5004580D5005584B
:104990000E5006580F50075810500858D8A0D3EFA3
:1049A000A4F0D5EFA4F0E6EFA4F00950015E0A50A0
:1049B000025A0B50035A0C50045A0D50055A0E500F
:1049C000065A0F50075A1050085A1380D8901032C8
:1049D0000F320E320D320C320B320A320932112EE6
:1049E000B5EFA4F01250D8B4F8EFA4F0FAEFA4F0A9
:1049F0000AEFA5F01A1E191E181E171E161E151EE8
:104A0000141E136C000E14221522162217221822CF
:104A100019221A2213C001F014C002F015C003F0CD
:104A200016C004F017C005F018C006F019C007F052
:104A30001AC008F01200000E116E000E106E000E6B
:104A40000F6E000E0E6E27EFA5F0084A092A6000CF
:104A500023F0F6FF600027F0F7FF000EF86E080065
:104A6000F550200AD8B437EFA5F039EFA5F025EFBF
:104A7000A5F0F70E0A6EFF0E0B6E600023F0F6FF36
:104A8000600027F0F7FF000EF86E0800F5500C6E7E
:104A90000D6A0A500C260B500D220D5009E1050E2F
:104AA0000C5CD8A056EFA5F058EFA5F025EFA5F0C7
:104AB00062EFA5F0000E0F6E010E0E6E084A092A75
:104AC0009FEFA5F0600023F0F6FF600027F0F7FFEE
:104AD000000EF86E0800F5500A6E0B6A0B50000AC3
:104AE000D8B475EFA5F09FEFA5F00A502B0AD8B403
:104AF0005EEFA5F0060AD8B45AEFA5F09FEFA5F037
:104B000010C001F011C002F0000E046E0A0E036E18
:104B100000ECBAF0600023F0F6FF600027F0F7FF2A
:104B2000000EF86E0800F550015E000E025A300EBD
:104B30000124106E000E0220116E5EEFA5F0D00E63
:104B40000A6EFF0E0B6E600023F0F6FF600027F088
:104B5000F7FF000EF86E0800F5500C6E0D6A0A5053
:104B60000C260B500D220D5009E10A0E0C5CD8A04A
:104B7000BCEFA5F0BEEFA5F080EFA5F00E500F1032
:104B8000D8A4C5EFA5F0C7EFA5F0D5EFA5F010C0EC
:104B90000AF011C00BF00A1E0B1E0A4A0B2A0AC0AB
:104BA00008F00BC009F0D9EFA5F010C008F011C053
:104BB00009F01200000E126E08BEE3EFA5F0E1EF5F
:104BC000A5F0F5EFA5F0081E071E061E051E041E23
:104BD000031E021E016C000E022203220422052283
:104BE000062207220822010E126E10BEFCEFA5F06D
:104BF000FAEFA5F00CEFA6F0101E0F1E0E1E0D1EF4
:104C00000C1E0B1E0A1E096C000E0A220B220C221F
:104C10000D220E220F22102209500A100B100C1028
:104C20000D100E100F101010D8B419EFA6F01BEFD6
:104C3000A6F063EFA6F0010E116E29EFA6F0D89052
:104C400009360A360B360C360D360E360F36103650
:104C5000112A10AE2EEFA6F030EFA6F01FEFA6F04F
:104C60000950015C0A5002580B5003580C5004586C
:104C70000D5005580E5006580F5007581050085840
:104C8000D8A045EFA6F047EFA6F057EFA6F00950E1
:104C9000015E0A50025A0B50035A0C50045A0D5030
:104CA000055A0E50065A0F50075A1050085AD890FD
:104CB00010320F320E320D320C320B320A32093200
:104CC000112E30EFA6F01250D8B469EFA6F06BEFBA
:104CD000A6F07BEFA6F0081E071E061E051E041E8A
:104CE000031E021E016C000E022203220422052272
:104CF00006220722082201C001F002C002F003C010
:104D000003F004C004F005C005F006C006F007C0BB
:104D100007F008C008F0120001C008F002C009F056
:104D200003C00AF004C00BF00506D8A0060605284B
:104D300006E10628D8A49FEFA6F0A1EFA6F0AEEFFB
:104D4000A6F0000E026E000E016E34EFA7F0084AC6
:104D5000092A0A4A0B2A0506D8A00606600023F095
:104D6000F6FF600027F0F7FF000EF86E1F0EF764E5
:104D700003D00800F55007D06F00DBFFE9FF6F009C
:104D8000DFFFEAFFEF500009D8B4C9EFA6F0CBEF80
:104D9000A6F00FEFA7F060002BF0F6FF60002FF0F9
:104DA000F7FF000EF86E0800F5500009D8B4DBEFED
:104DB000A6F0DDEFA6F00FEFA7F005500610D8B46F
:104DC000E4EFA6F0E6EFA6F00FEFA7F060002BF0FF
:104DD000F6FF60002FF0F7FF000EF86E08006F007E
:104DE000D4FF07F0600023F0F6FF600027F0F7FF24
:104DF000000EF86E1F0EF76403D00800F55007D0C0
:104E00006F00DBFFE9FF6F00DFFFEAFFEF500718DD
:104E1000D8B40DEFA7F00FEFA7F0A7EFA6F0600052
:104E200023F0F6FF600027F0F7FF000EF86E1F0E6C
:104E3000F76403D00800F55007D06F00DBFFE9FFEF
:104E40006F00DFFFEAFFEF50076E60002BF0F6FF08
:104E500060002FF0F7FF000EF86E0800F550075CB9
:104E6000016E026AD8A002061200F40E076EFF0E51
:104E7000086EC5ECB5F0000E1D6E300E0DECB1F0F5
:104E8000680E216EE40EE82EFED7212EFCD700D04E
:104E9000320E87ECBAF0000E1D6E300E0DECB1F044
:104EA000150E216EC60EE82EFED7212EFCD700D09F
:104EB000330E87ECBAF0000E1D6E300E0DECB1F023
:104EC000150E216EC60EE82EFED7212EFCD700D07F
:104ED000340E87ECBAF0000E1D6E250E0DECB1F00D
:104EE000150E216EC60EE82EFED7212EFCD700D05F
:104EF000350E87ECBAF0010E1D6E280E0DECB1F0E8
:104F0000150E216EC60EE82EFED7212EFCD700D03E
:104F1000360E87ECBAF0010E1D6E080E0DECB1F0E6
:104F2000150E216EC60EE82EFED7212EFCD700D01E
:104F3000370E87ECBAF0010E1D6E010E0DECB1F0CC
:104F4000030E226E080E216E770EE82EFED7212E5C
:104F5000FCD7222EFAD700F0380E87ECBAF0010EFB
:104F60001D6E060E0DECB1F0150E216EC60EE82E6C
:104F7000FED7212EFCD700D0390E87ECBAF0010EF7
:104F80001D6E0C0E0DECB1F0150E216EC60EE82E46
:104F9000FED7212EFCD700D0410E87ECBAF01200CC
:104FA00003ECBBF00009D8B4D8EFA7F0DAEFA7F014
:104FB00016EFA8F0E7EFA7F051ECBBF062EFA8F016
:104FC000AAECBBF062EFA8F0000E62EFA8F018C1E7
:104FD0000CF019C10DF020EE09F102D8FAEFA7F09C
:104FE0000500FA6EDE50FD6EDE50FE6EDE50FF6E86
:104FF000FA5012000E6E0F6A0F50000AD8B403EF79
:10500000A8F0E4EFA7F00E50010AD8B4E4EFA7F03F
:10501000030AD8B4DCEFA7F0010AD8B4E0EFA7F098
:10502000070AD8B4E4EFA7F0E4EFA7F0F8ECBAF081
:105030000009D8B41EEFA8F020EFA8F061EFA8F0A7
:1050400001012951030B0009D8B429EFA8F02BEF77
:10505000A8F037EFA8F0010E0E6E2951030B0F6E6A
:105060000E500F5E29510F18FC0B0F18296F6000AE
:105070008FF4D9FF600093F4DAFFDF50126E234BF8
:10508000242B2507D8A0260725512611D8A44BEF9D
:10509000A8F04DEFA8F055EFA8F090ECB1F00E6E2F
:1050A0000E50106E116A59EFA8F0000E116E030E2B
:1050B000106E10C013F0125064ECBBF0135062EF8E
:1050C000A8F0030E12001CECB8F0330E18ECB9F087
:1050D000000E5D6E9A0E5D24D96EDA6A010EDA2238
:1050E00058ECB8F0DF6E5D2A070E5D647AEFA8F029
:1050F0007CEFA8F06AEFA8F0280E01019A19D8A455
:1051000084EFA8F086EFA8F08CEFA8F0D60E076E1B
:10511000FC0E086EC5ECB5F05E0E076EFF0E086E55
:10512000C5ECB5F07B0E87ECBAF0000E5D6E700E2C
:105130000001B66F020EB76FD90EB86FFF0EB96FD0
:105140009A0E5D24D96EDA6A010EDA22DF505B6EA8
:105150005B50BA6FBB6B80ECB4F0700E016E020E48
:10516000026EA7ECB3F0070E5D60B9EFA8F0BBEFDD
:10517000A8F0BEEFA8F02C0E87ECBAF05D2A070E5F
:105180005D64C5EFA8F0C7EFA8F097EFA8F07D0E1B
:1051900087ECBAF090ECB9F09A0E016E010E026E37
:1051A000070E036EFCECB2F05C6E700E0001B66F81
:1051B000020EB76F170EB86FFF0EB96F5CC0BAF072
:1051C000BB6B80ECB4F0700E016E020E026EA7ECA9
:1051D000B3F090ECB9F01200033404340A6E0A50B4
:1051E000D8A4F5EFA8F0F7EFA8F001EFA9F0000EB2
:1051F000016E000E026E000E036E000E046E6EEF66
:10520000A9F001C005F002C006F003C007F004C019
:1052100008F0200E11EFA9F0D890083207320632BC
:105220000532E82E0CEFA9F00550096E038EFF0E33
:105230000116FF0E0216FF0E0316000E0416960E40
:105240000A5E0ABE28EFA9F026EFA9F03EEFA9F00A
:105250000A50800A970FD8B030EFA9F032EFA9F0CA
:1052600034EFA9F0F7EFA8F0D890043203320232FD
:1052700001320A3E34EFA9F056EFA9F01F0E0A647E
:1052800044EFA9F046EFA9F04EEFA9F0F7EFA8F030
:10529000D89001360236033604360A060A50D8A4DE
:1052A00054EFA9F056EFA9F048EFA9F00950D8B48F
:1052B0005CEFA9F05EEFA9F066EFA9F0041E031EF3
:1052C000021E016C000E02220322042201C001F022
:1052D00002C002F003C003F004C004F01200000E8C
:1052E0002814306E000E2914316E800E2A14326E8E
:1052F0007F0E2B14336E3050311032103310D8A47F
:1053000084EFA9F086EFA9F08EEFA9F0000E286EC9
:10531000000E296E000E2A6E000E2B6E000E2C144D
:10532000306E000E2D14316E800E2E14326E7F0EF4
:105330002F14336E3050311032103310D8A4A3EF35
:10534000A9F0A5EFA9F0ADEFA9F0000E2C6E000EAC
:105350002D6E000E2E6E000E2F6E2BAEB2EFA9F04A
:10536000B4EFA9F0BDEFA9F0286C291ED8B0292A06
:105370002A1ED8B02A2A800E2B562FAEC2EFA9F0D3
:10538000C4EFA9F0CDEFA9F02C6C2D1ED8B02D2ABA
:105390002E1ED8B02E2A800E2F56000E281A000E70
:1053A000291A000E2A1A800E2B1A000E2C1A000E33
:1053B0002D1A000E2E1A800E2F1A2C50285C2D50FC
:1053C00029582E502A582F502B58D8B0EAEFA9F060
:1053D000ECEFA9F0EFEFA9F0D890F0EFA9F0D880AA
:1053E00012004EC10BF04FC10CF050C10DF051C175
:1053F0000EF001C00BF002C00CF003C00DF004C0B1
:105400000EF00BC005F00CC006F00DC007F00EC08A
:1054100008F0180E11EFAAF0D890083207320632C1
:105420000532E82E0CEFAAF00550096E0A6A095001
:105430000A10D8A41EEFAAF020EFAAF040EFAAF0BD
:10544000D8900B34056E0C34066E0D34076E0E3496
:10545000086E0550061007100810D8A432EFAAF005
:1054600034EFAAF03AEFAAF0000E026E020E016EBF
:105470006FEFAAF0000E026E030E016E6FEFAAF03E
:1054800009280A10D8A447EFAAF049EFAAF06BEF59
:10549000AAF00BC005F00CC006F00DC007F00EC05E
:1054A00008F0090ED8900536063607360836E82E7D
:1054B00052EFAAF00550061007100810D8B463EF99
:1054C000AAF066EFAAF0010E67EFAAF0000E016ED7
:1054D000026A6FEFAAF0000E026E040E016E120057
:1054E00020EE11F0070EDE6AE806FDE209500A1010
:1054F0000B100C100D100E100F101010D8B483EFFD
:10550000AAF085EFAAF0D7EFAAF0010E196E93EF7B
:10551000AAF0D89009360A360B360C360D360E3600
:105520000F361036192A10AE98EFAAF09AEFAAF0AB
:1055300089EFAAF0D8901136123613361436153684
:105540001636173618360950015C0A5002580B50AF
:1055500003580C5004580D5005580E5006580F5063
:10556000075810500858D8A0B8EFAAF0BAEFAAF020
:10557000CBEFAAF00950015E0A50025A0B50035AB1
:105580000C50045A0D50055A0E50065A0F50075A27
:105590001050085A1180D89010320F320E320D324E
:1055A0000C320B320A320932192E9AEFAAF011C0CE
:1055B00001F012C002F013C003F014C004F015C0D3
:1055C00005F016C006F017C007F018C008F012006A
:1055D0003132333435363738393031323334353689
:1055E00000313233343536373839303132333435AF
:1055F000360031323334353637383930313233349E
:10560000353600313233343536373839303132338C
:10561000343536003132333435363738393031327B
:10562000333435360031323334353637383930316A
:105630003233343536003132333435363738393059
:105640003132333435360031323334353637383948
:105650003031323334353600313233343536373841
:105660003930313233343536003132333435363730
:10567000383930313233343536003132333435361F
:10568000373839303132333435360031323334350E
:1056900036373839303132333435360031323334FD
:1056A00035363738393031323334353600313233EC
:1056B000343536373839303132333435360020EE30
:1056C0002EF0080EDE6AE806FDE21CECB8F0550E7E
:1056D00018ECB9F0000E3B6E3B502824D96E000E3A
:1056E0002920DA6EDF5018ECB9F03B2A070E3B6434
:1056F0007CEFABF07EEFABF06CEFABF0BE0E18ECD6
:10570000B9F0000E3B6E2E0E3B24D96EDA6A000E05
:10571000DA2258ECB8F0DF6E3B2A010E3B6493EFBF
:10572000ABF095EFABF083EFABF01CECB8F02E5084
:105730002FC02CF02D6A2CC02DF02C6A2C26000EC8
:105740002D222CC001F02DC002F0000E02BEFF0E73
:10575000036E046E010EA9ECA2F001C00FF002C0AE
:1057600010F003C011F004C012F0000E136E000E12
:10577000146E800E156E3D0E166ECEEC94F00FC0BA
:1057800037F010C038F011C039F012C03AF037C00D
:1057900028F038C029F039C02AF03AC02BF01200A6
:1057A0000001CC51CD11D8A4D8EFABF0DAEFABF0BB
:1057B000E0EFABF0CCC010F0CDC011F0E6EFABF0F5
:1057C000FF0ECC25106EFF0ECD21116ED0A1EBEF98
:1057D000ABF0EDEFABF0F6EFABF00CC001F0026A0E
:1057E0000AC003F00BC004F03CECACF011BEFBEFC0
:1057F000ABF0FDEFABF0FFEFABF003EFACF0000E62
:10580000116E000E106E000E0F6E000E0E6E15EF74
:10581000ACF0000E026E200E016E0AC003F00BC049
:1058200004F03CECACF00E4A0F2A10500E5C0F5006
:10583000800A0D6E1150800A0D58D8A022EFACF0EE
:1058400024EFACF009EFACF00001D0B12AEFACF0DE
:105850002CEFACF035EFACF00CC001F0026A0AC0DE
:1058600003F00BC004F03CECACF0010E0E240A6E09
:10587000000E0F200B6E120003500410D8B443EF3B
:10588000ACF045EFACF04EEFACF003500410D8A4F0
:105890004CEFACF04EEFACF053EFACF00150B0EC8D
:1058A000BBF0A7EFACF020EE09F00350D92604506E
:1058B000DA22DE50DE10D8B460EFACF062EFACF06C
:1058C0007DEFACF020EE09F00350D9260450DA2227
:1058D00010EE03F00350E1260450E222DE50E65CB5
:1058E000E650800A096EDE50800A0958D8B07BEF76
:1058F000ACF07DEFACF0A7EFACF020EE03F003507E
:10590000D9260450DA226F0078FF05F06F0074FF8B
:1059100006F060000FF0D9FF600013F0DAFF6F00AF
:1059200078FF07F06F0074FF08F005500724D96E68
:1059300006500820DA6E600007F0DFFF20EE03F06B
:105940000350D9260450DA22DE2A000EDD2212008E
:1059500009500A100B100C100D100E100F10101023
:10596000D8B4B5EFACF0B7EFACF0FFEFACF0010E90
:10597000116EC5EFACF0D89009360A360B360C36EE
:105980000D360E360F361036112A10AECAEFACF0B7
:10599000CCEFACF0BBEFACF00950015C0A50025800
:1059A0000B5003580C5004580D5005580E50065813
:1059B0000F50075810500858D8A0E1EFACF0E3EFB3
:1059C000ACF0F3EFACF00950015E0A50025A0B50F4
:1059D000035A0C50045A0D50055A0E50065A0F50D7
:1059E000075A1050085AD89010320F320E320D322A
:1059F0000C320B320A320932112ECCEFACF001C05E
:105A000001F002C002F003C003F004C004F005C0BE
:105A100005F006C006F007C007F008C008F0120045
:105A20000001D0A116EFADF018EFADF022EFADF010
:105A300013C00AF014C00BF011C00CF012C00DF02E
:105A4000BBECB7F016BE27EFADF029EFADF02FEFAE
:105A5000ADF015C01AF016C01BF033EFADF0000E1C
:105A60001B6E000E1A6E000E196E000E186E45EFBA
:105A7000ADF0000E026E200E016E11C003F012C0D8
:105A800004F03CECACF0184A192A1A50185C195072
:105A9000800A176E1B50800A1758D8A052EFADF03D
:105AA00054EFADF039EFADF00001D0B15AEFADF0E9
:105AB0005CEFADF066EFADF013C00AF014C00BF070
:105AC00011C00CF012C00DF0BBECB7F013C001F028
:105AD00014C002F099ECB5F01A500124116E1B505D
:105AE0000220126E1200000E066E04BE7CEFADF0B6
:105AF0007AEFADF082EFADF0036C041ED8B0042A4B
:105B0000010E066E02BE89EFADF087EFADF08FEFAC
:105B1000ADF0016C021ED8B0022A010E061A000E6A
:105B2000086E000E076E03500410D8B49AEFADF063
:105B30009CEFADF0C4EFADF0010E056EA4EFADF03B
:105B4000D89003360436052A04AEA9EFADF0ABEFCA
:105B5000ADF0A0EFADF0D890073608360350015CE9
:105B600004500258D8A0B7EFADF0B9EFADF0BEEFDA
:105B7000ADF00350015E0450025A0780D890043201
:105B80000332052EABEFADF00650D8B4CAEFADF03E
:105B9000CCEFADF0D0EFADF0076C081ED8B0082AFE
:105BA00007C001F008C002F012000FEFAEF0800E47
:105BB000C2ECB2F0510E1F6EF70E206E4FECB1F03A
:105BC000800EC2ECB2F02DEFAEF0C00EC2ECB2F01F
:105BD000510E1F6EF70E206E4FECB1F0C00EC2ECEE
:105BE000B2F02DEFAEF0940EC2ECB2F0500E1F6E7C
:105BF000FD0E206E4FECB1F0940EC2ECB2F02DEF22
:105C0000AEF0D40EC2ECB2F0500E1F6EFD0E206E40
:105C10004FECB1F0D40EC2ECB2F02DEFAEF024C0D8
:105C200026F025C027F02750000AD8B41AEFAEF0AE
:105C30002DEFAEF02650010AD8B4D7EFADF0030A2D
:105C4000D8B4E5EFADF0010AD8B4F3EFADF0070A30
:105C5000D8B401EFAEF02DEFAEF0D00E266ECA0E26
:105C6000E82EFED7262EFCD71200D00EF66E550E6B
:105C7000F76E010EF86E01EE00F010EEEEF0090086
:105C80006F00D7FFEEFFE550E150F9E1FA0EF66E36
:105C90006F0EF76E010EF86E00EEA6F110EE3DF0FD
:105CA00009006F00D7FFEEFFE550E150F9E10E0E5D
:105CB000F66E770EF76E010EF86E00EEFAF010EE4B
:105CC00006F009006F00D7FFEEFFE550E150F9E163
:105CD00000EE00F310EE00F1EE6AE550E150FCE159
:105CE000E250FAE100EE00F2C00EEE6AE806FDE1D5
:105CF00000EE00F1A60EEE6AE806FDE100EEC8F047
:105D0000320EEE6AE806FDE15F6A080ED56E000EFF
:105D1000D66E000ED76E000100EF80F0000E066E0A
:105D200002BE97EFAEF095EFAEF09DEFAEF0016CD6
:105D3000021ED8B0022A010E066E04BEA4EFAEF019
:105D4000A2EFAEF0A8EFAEF0036C041ED8B0042AA8
:105D500003500410D8B4AFEFAEF0B1EFAEF0D5EF12
:105D6000AEF0010E056EB9EFAEF0D89003360436F2
:105D7000052A04AEBEEFAEF0C0EFAEF0B5EFAEF068
:105D80000350015C04500258D8A0C9EFAEF0CBEF2D
:105D9000AEF0CFEFAEF00350015E0450025AD8903F
:105DA00004320332052EC0EFAEF00650D8B4DBEF5C
:105DB000AEF0DDEFAEF0E1EFAEF0016C021ED8B058
:105DC000022A01C001F002C002F01200000E01140C
:105DD000096E000E02140A6E800E03140B6E7F0E05
:105DE00004140C6E09500A100B100C10D8A4FBEF11
:105DF000AEF0FDEFAEF005EFAFF0000E016E000E5D
:105E0000026E000E036E000E046E000E0514096E85
:105E1000000E06140A6E800E07140B6E7F0E081417
:105E20000C6E09500A100B100C10D8A41AEFAFF02A
:105E30001CEFAFF024EFAFF0000E056E000E066E03
:105E4000000E076E000E086E055001180FE1065097
:105E500002180CE10750031809E108500418D8B4DF
:105E600034EFAFF036EFAFF039EFAFF0D8903AEF54
:105E7000AFF0D8801200016E010E026E010129B749
:105E800044EFAFF046EFAFF08BEFAFF001C022F17F
:105E900029952987FC0E29170F0E276F010E216FF8
:105EA000F40E206F29895C0E006F770E016F010ED2
:105EB000026F000E126F000E136F5C0E036F770EF1
:105EC000046F010E056F000E146F000E156F5C0E4F
:105ED000066F770E076F010E086F000E166F000E2B
:105EE000176F5C0E096F770E0A6F010E0B6F000EB5
:105EF000186F000E196F580E0C6F770E0D6F010E94
:105F00000E6F000E1A6F000E1B6F83ECBBF0A7EC38
:105F1000B9F0000E026E0250120001012989B1EFA2
:105F2000AFF099ECBBF0080EDEEFAFF099ECBBF0F0
:105F3000070EDEEFAFF00101252969ECBBF0040E7E
:105F4000DEEFAFF0070E01012719D8B4AAEFAFF0CA
:105F5000ACEFAFF0AEEFAFF09CECBBF00F0EDEEFAE
:105F6000AFF012C10CF013C10DF002D8C2EFAFF0C8
:105F70000500FA6E0051FD6E0151FE6E0251FF6E7A
:105F8000FA5012000E6E0F6A0F50000AD8B4CBEF11
:105F9000AFF0A2EFAFF00E50010AD8B4A2EFAFF00D
:105FA000030AD8B496EFAFF0010AD8B491EFAFF07E
:105FB000070AD8B49BEFAFF0A2EFAFF012000EECDF
:105FC000BBF00009D8A4E7EFAFF0E9EFAFF0ECEFDA
:105FD000AFF0040E2DEFB0F001012951030B0009C1
:105FE000D8B4F5EFAFF0F7EFAFF003EFB0F0010E7C
:105FF000106E2951030B116E1050115E29511118AA
:10600000FC0B1118296F2507D8A02607255126114A
:10601000D8B40DEFB0F00FEFB0F01DEFB0F096EC8C
:10602000BBF060008FF4D9FF600093F4DAFFDF6EFD
:106030000101234B242BE9EFAFF08DECAFF0126E92
:1060400096ECBBF060008FF4D9FF600093F4DAFFA8
:10605000DF6E0101234B242B125012003901A3A73C
:1060600034EFB0F036EFB0F07AEFB0F093A73BEF3B
:10607000B0F03DEFB0F07AEFB0F06F00A0F7F9F0BC
:106080000D0E0001F919D8B448EFB0F04AEFB0F0A6
:1060900055EFB0F0E35109E1800EE25DD8A053EF77
:1060A000B0F055EFB0F06BEFB0F0010EF46F000EF2
:1060B000E225D96E030EE321DA6E000EDF6EE2C038
:1060C0008AF1E3C08BF1000EE36F000EE26F39013D
:1060D00093977AEFB0F0000EE225D96E030EE3211C
:1060E000DA6E6000E7F3DFFFE24BE32BE2C08AF1F8
:1060F000E3C08BF1110022500001FA5DFB51800AD0
:10610000256E2350800A2558D8B089EFB0F08BEF68
:10611000B0F08FEFB0F0FAC022F0FBC023F0200403
:106120002110D8A496EFB0F098EFB0F09CEFB0F04B
:1061300022507F0FC2ECB2F0020E20182110D8A41A
:10614000A4EFB0F0A6EFB0F0AAEFB0F02250BF0F6E
:10615000C2ECB2F0030E266E080E256E770EE82E06
:10616000FED7252EFCD7262EFAD700F024500DECB2
:10617000B2F0030E266E080E256E770EE82EFED7BF
:10618000252EFCD7262EFAD700F01200066E0150FD
:1061900002100310D8B4CFEFB0F0D1EFB0F0F2EFAF
:1061A000B0F00650030D000EF324D96E010EF4205A
:1061B000DA6E600007F0DEFF60000BF0DEFF6000CB
:1061C0000FF0DEFF0650020D120EF324D96E010E01
:1061D000F420DA6E600013F0DEFF600017F0DDFFE0
:1061E0000CEFB1F00650030D000EF324D96E010E32
:1061F000F420DA6E5C0EDE6E770EDE6E010EDE6E61
:106200000650020D120EF324D96E010EF420DA6E40
:10621000000EDE6E000EDD6E12001F6E1F50F00BC2
:106220000C09206E20C01BF05F5015ECBAF0500E28
:10623000E82EFED71F50F00B0809206E20C01BF07F
:106240005F5015ECBAF0500EE82EFED71D04D8A40E
:106250002CEFB1F02EEFB1F04EEFB1F01FC01EF0F9
:106260000F0E1E161E38F00B0C09206E20C01BF0FE
:106270005F5015ECBAF0500EE82EFED71FC01EF08E
:106280000F0E1E161E38F00B0809206E20C01BF0E2
:106290005F5015ECBAF0500EE82EFED71200000E3B
:1062A000236E000E226E6DEFB1F060007FF0F6FFFE
:1062B000600083F0F7FF000EF86E0800F5500DEC5B
:1062C000B2F01F4A202A224A232A150E216EC60E3A
:1062D000E82EFED7212EFCD700D060007FF0F6FF1D
:1062E000600083F0F7FF000EF86E0800F55000091B
:1062F000D8B47DEFB1F07FEFB1F08FEFB1F00001D6
:10630000FA51225C2350800A216EFB51800A2158E9
:10631000D8A08DEFB1F08FEFB1F055EFB1F01200D2
:1063200001012989A5EFB1F099ECBBF0070ECEEF82
:10633000B1F00101252969ECBBF0030ECEEFB1F0FD
:106340009CECBBF00A0ECEEFB1F012C10CF013C101
:106350000DF002D8B6EFB1F00500FA6E0051FD6EF7
:106360000151FE6E0251FF6EFA5012000E6E0F6A5E
:106370000F50000AD8B4BFEFB1F0A0EFB1F00E504B
:10638000010AD8B4A0EFB1F0030AD8B494EFB1F089
:10639000060AD8B499EFB1F0A0EFB1F01200000EE8
:1063A000BA6E000EBB6E000EBC6E000EC26EC368ED
:1063B000A70EC46E000E3A01606F000E506F000E03
:1063C000406F000E816F7F0E516F4169C00E616F8B
:1063D000000E5A6F000E5B6F070E426F000E526F79
:1063E000180E626F4369536963694469546964694B
:1063F000080E846F000E476F000E466F000E456F4B
:10640000140EE26F210E136F220E146F130E166F0F
:10641000170EE56F130EE16F12001E6E1E50F00B8B
:106420000D090001EC6FECC01BF05F5015ECBAF0E9
:10643000500EE82EFED71E50F00B09090001EC6F3C
:10644000ECC01BF05F5015ECBAF0500EE82EFED7F2
:106450001EC01DF00F0E1D161D38F00B0D0900019A
:10646000EC6FECC01BF05F5015ECBAF0500EE82E4C
:10647000FED71EC01DF00F0E1D161D38F00B0909AA
:106480000001EC6FECC01BF05F5015ECBAF0500E41
:10649000E82EFED71200246E2050216E226A215071
:1064A0000001FA5DFB51800A236E2250800A2358B6
:1064B000D8B05DEFB2F05FEFB2F061EFB2F0FA0585
:1064C000206E2404D8A467EFB2F069EFB2F06DEF4C
:1064D000B2F020507F0FC2ECB2F0020E2418D8A404
:1064E00074EFB2F076EFB2F07AEFB2F02050BF0F57
:1064F000C2ECB2F0020E226EA00E216E920EE82EB9
:10650000FED7212EFCD7222EFAD700D0120083EC22
:10651000BBF0020E0101286F9AEFB2F051ECBBF014
:10652000C1EFB2F0AAECBBF0C1EFB2F042ECBBF0AD
:10653000C1EFB2F014C10CF015C10DF020EE03F163
:1065400002D8ADEFB2F00500FA6EDE50FD6EDE50FF
:10655000FE6EDE50FF6EFA5012000E6E0F6A0F5084
:10656000000AD8B4B6EFB2F096EFB2F00E50020ABD
:10657000D8B48EEFB2F0010AD8B492EFB2F096EF31
:10658000B2F012001E6E1E50F00B0C091F6E1FC0E1
:106590001BF05F5015ECBAF0500EE82EFED71E50DF
:1065A000F00B08091F6E1FC01BF05F5015ECBAF00E
:1065B000500EE82EFED71EC01DF00F0E1D161D3802
:1065C000F00B0C091F6E1FC01BF05F5015ECBAF0EA
:1065D000500EE82EFED71EC01DF00F0E1D161D38E2
:1065E000F00B08091F6E1FC01BF05F5015ECBAF0CE
:1065F000500EE82EFED71200000E046E000E086E3C
:10660000000E066E2AEFB3F006500124D96E000E7C
:106610000220DA6EDF50056E000E076E0850051876
:10662000010B046ED89008320450D8B41AEFB3F0BE
:106630001CEFB3F01EEFB3F08C0E081AD8900532A1
:10664000072A070E076427EFB3F029EFB3F00EEF28
:10665000B3F0062A0350065CD8A031EFB3F033EF55
:10666000B3F004EFB3F00850120060000FF0F6FF33
:10667000600013F0F7FF000EF86E08006F00D4FF03
:10668000EBF05CEFB3F060000FF0F6FF600013F08A
:10669000F7FF000EF86E08006F00D4FFEBF060000B
:1066A00007F0D9FF60000BF0DAFF6000AFF3DFFF07
:1066B000014A022A034A042A0001EB51D8A463EFDD
:1066C000B3F065EFB3F043EFB3F0600007F0D9FF2C
:1066D00060000BF0DAFF000EDF6E120095ECB6F0F2
:1066E00001012951030B0009D8B479EFB3F07BEF16
:1066F000B3F088EFB3F003ECBBF00009D8B483EF3C
:10670000B3F085EFB3F088EFB3F0100E0101276FFF
:1067100001012751030D050EF324F66EF50EF4204A
:10672000F76EF86A000EF82202D8A4EFB3F0050065
:10673000FA6E0900F550FD6E0900F550FE6E090075
:10674000F550FF6EFA5012000101276F1200000E83
:10675000046E000E036ED0EFB3F03901A3A9B3EFBE
:10676000B3F0B5EFB3F0ADEFB3F003500124D96E41
:1067700004500220DA6EDF503D01EA6F034A042A1A
:1067800004BECCEFB3F0045009E1810E035CD8A045
:10679000CCEFB3F0CEEFB3F0D0EFB3F0DEEFB3F069
:1067A00003500124D96E04500220DA6EDF50D8A4C1
:1067B000DCEFB3F0DEEFB3F0ADEFB3F01200FC0EA0
:1067C00001012917020E286F2995EEEFB3F0A8EC0E
:1067D000BBF015EFB4F00F0E15EFB4F016C10CF0CE
:1067E00017C10DF020EE06F102D801EFB4F005005C
:1067F000FA6EDE50FD6EDE50FE6EDE50FF6EFA5019
:1068000012000E6E0F6A0F50000AD8B40AEFB4F0EF
:10681000EBEFB3F00E50020AD8B4E7EFB3F0010A81
:10682000D8B4E7EFB3F0EBEFB3F01200B2C04AF028
:10683000B3C04BF0000E0101636F000E626F34EFC6
:10684000B4F0B0C040F0B1C041F04A0E426E000E4C
:10685000436EB4C044F0B5C045F090EC8CF04050AD
:10686000010162274150632360002BF1F6FF6000B5
:106870002FF1F7FF000EF86E0800F5500009D8A4BC
:1068800044EFB4F046EFB4F021EFB4F062C1B0F0E1
:1068900063C1B1F0120007C00BF008C00CF005C0D6
:1068A0000DF006C00EF00B50096E0C500A6E0B4A2C
:1068B0000C2A600027F0F6FF60002BF0F7FF000EB7
:1068C000F86E600037F0D9FF60003BF0DAFF0D4A48
:1068D0000E2A1F0EF76403D00800F55007D06F0092
:1068E000DBFFE9FF6F00DFFFEAFFEF50DF6EDF50F5
:1068F000D8A47DEFB4F07FEFB4F053EFB4F0120002
:10690000BA0E4E6E000E4F6EB6C050F0B7C051F0CA
:10691000000E546E000E536E000E5A6E000E596E2D
:10692000500E0001B06F000EB16FB8C0B2F0B9C028
:10693000B3F04E0EB46F000EB56F16ECB4F0B0C0ED
:106940004CF0B1C04DF053500001B625D96E5450F3
:10695000B721DA6E000EDF6E4CC0B6F04DC0B7F056
:106960001200000E236E000E226EC2EFB4F0225011
:106970001F24D96E23502020DA6EDF500DECB2F0C8
:10698000224A232A22501F24D96E23502020DA6E57
:10699000DF50D8B4CEEFB4F0D0EFB4F0E0EFB4F005
:1069A0000001FA51225C2350800A216EFB51800ABB
:1069B0002158D8A0DEEFB4F0E0EFB4F0B7EFB4F0B8
:1069C00012001A6E1A503BECAFF00009D8B4EBEF8E
:1069D000B4F0EDEFB4F0E2EFB4F016C001F017C080
:1069E00002F018C003F019C004F064ECBAF0000E15
:1069F000076E000E086E000E096E000E0A6E000E85
:106A00000B6EC4ECBAF073ECBBF0D5ECB9F0E80651
:106A1000D8B40DEFB5F00FEFB5F005EFB5F01200FB
:106A20003901A3A116EFB5F018EFB5F01AEFB5F0E4
:106A30003DEFB5F0A2AF1FEFB5F021EFB5F023EFBA
:106A4000B5F03DEFB5F03D0179A529EFB5F02BEF9D
:106A5000B5F02DEFB5F03DEFB5F079AF32EFB5F011
:106A600034EFB5F036EFB5F03DEFB5F076A93BEF7A
:106A7000B5F03DEFB5F010EFB5F0120003C009F02E
:106A800004C00AF001C007F002C008F05DEFB5F0E5
:106A9000600027F0D9FF60002BF0DAFFDF500B6EAB
:106AA000094A0A2A60001FF0D9FF600023F0DAFFCC
:106AB00060002FF0DFFF074A082A0506D8A0060667
:106AC000052806E10628D8A468EFB5F06AEFB5F00E
:066AD00048EFB5F01200D2
:106AD8003901A9A172EFB5F074EFB5F098EFB5F0F0
:106AE80099A179EFB5F07BEFB5F098EFB5F000011B
:106AF800DDBF87EFB5F0DD5108E1DC05D8A087EFF1
:106B0800B5F089EFB5F08EEFB5F0DC07D8A0DD075A
:106B180091EFB5F0F28B39019991000E0101776F71
:106B2800010E766F3901A991110001C003F002C06E
:106B380004F0A1EFB5F0014A022A600007F0F6FF61
:106B480060000BF0F7FF000EF86E1F0EF76403D01D
:106B58000800F55007D06F00DBFFE9FF6F00DFFF8B
:106B6800EAFFEF500009D8A4BCEFB5F0BEEFB5F0CE
:106B78009FEFB5F00350015C016E04500258026E9D
:106B88001200DDEFB5F03901A3A9CDEFB5F0CFEFD5
:106B9800B5F0C7EFB5F060001FF0F6FF600023F016
:106BA800F7FF000EF86E08006F00D7FFEAFD074AEE
:106BB800082A60001FF0F6FF600023F0F7FF000EC0
:106BC800F86E0800F5500009D8A4EDEFB5F0EFEF26
:106BD800B5F0C7EFB5F01200046E000E01016F6F3B
:106BE800000E6E6F07EFB6F0520E026E2B0E016E9E
:106BF800000EE82EFED7012EFCD7022EFAD700D0C1
:106C080001016E4B6F2B0450016E026A01506E5DDC
:106C18006F51800A036E0250800A0358D8A017EFFC
:106C2800B6F019EFB6F0F8EFB5F01200000ED2BECC
:106C3800010E046E0250030B3901E16F600007F08A
:106C4800E0F960000FF0E3F93F0EE517E585D29E05
:106C5800550EE66FAA0EE66FE58334EFB6F000F046
:106C68003901E5B33AEFB6F03CEFB6F033EFB6F0E2
:106C7800E59504B002D0D29E01D0D28E1200010E4A
:106C8800076E200E01180210D8B44DEFB6F04FEF82
:106C9800B6F068EFB6F0F70E036EFF0E046E01C093
:106CA80005F002C006F003500526045006220650DF
:106CB80009E1050E055CD8A064EFB6F066EFB6F002
:106CC80068EFB6F0000E076E07C001F0026A120006
:106CD800146E010E156E010129B575EFB6F077EF48
:106CE800B6F093EFB6F02985000E156E255169ECC4
:106CF800BBF01450D8B483EFB6F085EFB6F08CEF44
:106D0800B6F0040E0101276FBEECB9F091EFB6F0B2
:106D1800030E0101276FEDECBAF0A6ECBAF015509E
:106D280012002FECBBF00009D8B49DEFB6F09FEF2E
:106D3800B6F0A3EFB6F0A5ECBBF0BDEFB6F019ECDA
:106D4800BBF00009D8B4ABEFB6F0ADEFB6F0B1EFD9
:106D5800B6F09FECBBF0BDEFB6F024ECBBF0000939
:106D6800D8B4B9EFB6F0BBEFB6F0BDEFB6F0A2EC11
:106D7800BBF0120020EE02F00C50D9260D50DA229A
:106D88006F0078FF01F06F0074FF02F0600033F0CD
:106D9800D9FF600037F0DAFF6F0078FF03F06F006B
:106DA80074FF04F064ECBAF0000E076E000E086E73
:106DB800000E096E000E0A6E000E0B6ED2ECBAF0D1
:106DC800020E1200010E0114016E026A0150021037
:106DD800D8B4F1EFB6F0F3EFB6F000EFB7F0C29029
:106DE800CA901A0EE82EFED700D0C280C00E00D07E
:106DF800E82EFDD70BEFB7F0C290CA90E00E00D096
:106E0800E82EFDD7C2800A0EE82EFED700D0120069
:106E1800000E3D01EC6F000EED6F000EEE6F000EE0
:106E2800EF6F000EF06F000EF16FB00EF26F800E74
:106E3800F36F000EF46F8A0EF56F000EF66F000EFA
:106E4800F76F000EF86F000EF96F000EFA6FF28BF5
:106E5800F289390193971200BF0E096EFF0E0A6E70
:106E680007C00BF008C00CF009500B260A500C2282
:106E78000C5007E11A0E0B5CD8B045EFB7F047EF9E
:106E8800B7F04EEFB7F0200E0710076E0850086EE7
:106E980052EFB7F007C007F008C008F01200000E64
:106EA8002C1A000E2D1A000E2E1A800E2F1A28C02A
:106EB80001F029C002F02AC003F02BC004F02CC056
:106EC80005F02DC006F02EC007F02FC008F06EECBC
:106ED80092F001C028F002C029F003C02AF004C0D3
:106EE8002BF01200026E800E036E90EFB7F0025086
:106EF80003140009D8B483EFB7F085EFB7F08AEF31
:106F0800B7F02A0E87ECBAF08DEFB7F0200E87ECB9
:106F1800BAF0D8900330036E0350D8A496EFB7F0B8
:106F280098EFB7F07BEFB7F012009F0E096EFF0ED7
:106F38000A6E07C00BF008C00CF009500B260A5067
:106F48000C220C5007E11A0E0B5CD8B0AEEFB7F06C
:106F5800B0EFB7F0B6EFB7F05F0E0714076E086A28
:106F6800BAEFB7F007C007F008C008F01200000E2B
:106F7800106E000E0F6ECCEFB7F00EC001F0026A73
:106F88000CC003F00DC004F03CECACF00F4A102A22
:106F98000F500A24D96E10500B20DA6EDF500E6E97
:106FA8000E50D8A4DAEFB7F0DCEFB7F0C1EFB7F0C6
:106FB800120014BEEAEFB7F0145006E11304D8B07B
:106FC800E8EFB7F0EAEFB7F0F8EFB7F013C015F055
:106FD80014C016F0151E161E154A162A15C013F0F1
:106FE80016C014F0FCEFB7F013C013F014C014F07F
:106FF80012004FF6A1F5AEF619F7FAF64EF538F786
:1070080082F6D6F664F70102030405060708286E1F
:10701800756C6C2900C0FF28FF47158116032428CA
:0F702800AA4265261302B628AA56C138140140A1
:10703800C290CA900A0E016EF80EE82EFED7012EF5
:10704800FCD700D0C280C00E00D0E82EFDD7CAB051
:1070580030EFB8F032EFB8F039EFB8F0E40E00D006
:1070680000D0E82EFCD700D000D012009F0E036E8F
:10707800FF0E046E200E0110056E000E0210066E43
:10708800035005260450062206500AE11A0E055C34
:10709800D8A051EFB8F054EFB8F0010E55EFB8F0A2
:1070A800000E016E026A1200000E026E000E036EE0
:1070B800D8900232EBECB9F00009D8B466EFB8F01A
:1070C80068EFB8F069EFB8F0028E032A070E036480
:1070D80070EFB8F072EFB8F05CEFB8F00250120041
:1070E8009F0E036EFF0E046E01C005F002C006F08D
:1070F800035005260450062206500AE11A0E055CC4
:10710800D8A089EFB8F08CEFB8F0010E8DEFB8F089
:10711800000E016E026A1200BF0E036EFF0E046EAF
:1071280001C005F002C006F00350052604500622EF
:1071380006500AE11A0E055CD8A0A5EFB8F0A8EF32
:10714800B8F0010EA9EFB8F0000E016E026A120045
:107158000150021003100410D8B4B5EFB8F0B7EF1F
:10716800B8F0BFEFB8F0000E011A000E021A000EB8
:10717800031A800E041A01C001F002C002F003C015
:1071880003F004C004F01200D00E036EFF0E046E6C
:1071980001C005F002C006F003500526045006227F
:1071A80006500AE10A0E055CD8A0DDEFB8F0E0EF62
:1071B800B8F0010EE1EFB8F0000E016E026A12009D
:1071C8000001DE51DF11D8A4ECEFB8F0EEEFB8F013
:1071D800F5EFB8F0B290390194910001F283F8EF1D
:1071E800B8F0DE07D8A0DF07CF0EB16E2C0EB06E58
:1071F8003901A49111003D017995600007F06EFDF9
:10720800000E6C6F738B79A50CEFB9F00EEFB9F027
:1072180007EFB9F074AB13EFB9F016EFB9F0010E40
:1072280017EFB9F0000E1200046E000E056E04C0D0
:1072380003F0010E03160350016E026AE6ECB6F085
:10724800D8900432052A070E05642DEFB9F02FEF08
:10725800B9F01BEFB9F012000CC001F00DC002F03C
:10726800000E046E010E036E64ECBAF0000E076E99
:10727800000E086E000E096E000E0A6E000E0B6EF0
:10728800D2ECBAF0040E12000CC001F00DC002F0EE
:10729800000E046E020E036E64ECBAF0000E076E68
:1072A800000E086E000E096E000E0A6E000E0B6EC0
:1072B800D2ECBAF0020E12000CC001F00DC002F0C0
:1072C800000E046E010E036E64ECBAF0000E076E39
:1072D800000E086E000E096E000E0A6E000E0B6E90
:1072E800D2ECBAF0020E12000CC001F00DC002F090
:1072F800000E046E020E036E64ECBAF0000E076E08
:10730800000E086E000E096E000E0A6E000E0B6E5F
:10731800D2ECBAF0040E12003901A3A996EFB9F025
:1073280098EFB9F090EFB9F00D0E3D01EA6F390111
:10733800A3A9A1EFB9F0A3EFB9F09BEFB9F00A0E3A
:107348003D01EA6F12003D0173BFADEFB9F0AFEF39
:10735800B9F0BDEFB9F0000E796F000E7A6F000E2C
:10736800766F6C69510E3A016A6F510E6B6F3D0171
:10737800738F120001012951FC0B0209296F2505A1
:107388002611D8A4CAEFB9F0CCEFB9F0CEEFB9F016
:107398008DECAFF0D8800101223564ECBBF0040E0F
:1073A8001200010E016E010129B5DDEFB9F0DFEF22
:1073B800B9F0E9EFB9F02997226983ECBBF0B5EC95
:1073C800BAF05EECBBF028C101F001501200C29087
:1073D800CA90050EE82EFED700F0C2801A0EE82EDD
:1073E800FED700D0000ECAB0010E016EB00E00D05C
:1073F800E82EFDD701501200015003026F00CCFFA8
:1074080005F06F00D0FF06F001500402F350062685
:1074180002500302F350062605C001F006C002F030
:1074280012001C6E1BC0A2F1000E0101A36FA20E78
:10743800166E010E176E000E196E010E186E1C5096
:10744800E1ECB4F0A00EE82EFED712008DECBBF0F4
:107458008AECBBF00009D8B434EFBAF036EFBAF0D2
:107468003CEFBAF0000E69ECBBF0000E64ECBBF028
:10747800000E12001CECB8F0CC0E18ECB9F0440E5B
:1074880018ECB9F0EBECB9F00009D8B44EEFBAF04B
:1074980050EFBAF046EFBAF012000FC001F010C07A
:1074A80002F099ECB5F001500F24056E025010203F
:1074B800066E11C007F012C008F04BECB4F01200D1
:1074C800010129A96AEFBAF06CEFBAF075EFBAF0CA
:1074D80001C023F102C024F103C025F104C026F144
:1074E80029991200030E3D017B6F040E736F800E05
:1074F800746F000E756F000E6C6F7599200E6E6FAD
:107508007995739F1200016E8BEFBAF000F0390184
:10751800A3A991EFBAF093EFBAF08AEFBAF060003E
:1075280007F0EAFD12000250030B3901E16F600019
:1075380007F0E0F93F0EE517E58100F000F03901AA
:10754800E3511200ACEFBAF010ECB5F06EECB3F00A
:10755800010129B5B2EFBAF0B4EFBAF0A8EFBAF06A
:107568001200390193939395929F93913D017A91DB
:107578007A957A9F7A9D7A9376937695769112008A
:1075880007C001F008C002F009C003F00AC004F007
:107598000BC005F0020EC6ECB0F0120007C001F0F7
:1075A80008C002F009C003F00AC004F00BC005F0DF
:1075B800000EC6ECB0F01200286E25C020F028504E
:1075C8004BECB2F026C01FF027C020F0B1ECB4F0AD
:1075D800120001012951FC0B0209296F22512225B1
:1075E80064ECBBF0030E12003D0178BBFEEFBAF06D
:1075F80001EFBBF0010E02EFBBF0000E12003D01DF
:1076080074BB09EFBBF00CEFBBF0010E0DEFBBF044
:10761800000E12003D0178B114EFBBF017EFBBF07C
:10762800010E18EFBBF0000E12003D0179B51FEFF7
:10763800BBF022EFBBF0010E23EFBBF0000E1200EF
:107648003D0176B92AEFBBF02DEFBBF0010E2EEF0E
:10765800BBF0000E12003D0179BF35EFBBF038EFEB
:10766800BBF0010E39EFBBF0000E12006EECBBF060
:1076780001012995020E286F0F0E12006EECBBF067
:1076880001012995000E286F0F0E120090ECBBF037
:107698008DECBBF058ECBBF012000101255169ECF0
:1076A800BBF0BEECB9F0120001012995000E286F5D
:1076B8000F0E12003D01739F000E796F788512003E
:1076C800016E600007F06BFD1200016E600007F0AC
:1076D8006CFD12003D01739F7885738F1200000EB8
:1076E8006CECB6F0120090ECBBF0090E120093ECB3
:1076F800BBF0040E120093ECBBF0030E1200000E58
:107708003D01796F120010000E140F133D016C51EA
:1077180012003D01739B12003D01748D12003D0162
:10772800749D12003D016A5112003D01738D1200D3
:107738003D01739D12003D01799512003D01769936
:1077480012003D01799F1200010E1200020E120074
:0A775800050E1200010E12001200CF
:020000040020DA
:10000000FF0FFF0FFF0FFF0FFF0FFF0FFF0FFF0F80
:020000040030CA
:0A0000008CD5FFF78DCFFFDFFFFF67
:020000040031C9
:10000000630000000000000000000000000000008D
:1000100028FF47158116032400000000000000009F
:1000200028AA4265261302B6000000000000000066
:1000300028AA56C13814014000000000000000004A
:1000400028AA0D82381401CD000000000000000035
:10005000630000000000000000000000000000003D
:1000600028FF47158116032400000000000000004F
:1000700028AA4265261302B6000000000000000016
:1000800028AA56C1381401400000000000000000FA
:1000900028AA0D82381401CD0000000000000000E5
:00000001FF
